:100000000C946D000C94BC000C94BC000C94BC00CF
:100010000C94BC000C94BC000C94DC1D0C94BC0033
:100020000C94BC000C94BC000C94BC000C94BC0060
:100030000C94BC000C94BC000C94BC000C94F31405
:100040000C94BC000C94BC000C9436190C949A19B6
:100050000C94BC000C94BC000C94BC000C94BC0030
:100060000C94BC000C94BC000C94BC000C94BC0020
:100070000C94BC000C94BC000C94BC000C94BC0010
:100080000C94BC000C94BC000C94BC00701F7C1F32
:100090008C1F971FAA1FAD1FB01FB31FB61FDB1FFA
:1000A0000C20492034205620142025203C204420B8
:1000B000632074206D1F6D1F6D1F6D1F84208920AC
:1000C0008C20A020AD20B9206D1FC620D120DE20BD
:1000D000E920F62001210E21192180EC85BF87E05F
:1000E00089B98093990011241FBECFEFD0E1DEBF04
:1000F000CDBF12E0A0E0B1E0EAE4F5E900E00BBF1B
:1001000002C007900D92AA37B107D9F713E0AAE70A
:10011000B2E001C01D92A138B107E1F78FEF9FE770
:100120009EBF8DBF8FEF9FE78158934081589140CC
:1001300040F06FEF7EE76158734081E893E00E94E2
:10014000D70C0E94F612892B59F0A7E4B3E0E3E63E
:10015000F1E089E001900D928150E1F70E94DD12FB
:1001600020E831E040E050E062EB7BE08CE691E09B
:100170000E9459130C9400000C94000060918002BE
:100180007091810299270E940D4908958091800203
:10019000909181020E94874899270895809180025A
:1001A000909181020E9487482FEF8F3F920749F07C
:1001B00060918002709181020E94FD4881E090E090
:1001C000089580E090E008950F931F93CF93DF93FD
:1001D0008C01EB010E941D06823061F0843019F41D
:1001E0000FC00E94C6000E94CE008823D1F780E095
:1001F00090E00BC0C8010E94930280E090E005C02F
:10020000BE01C8010E944F059927DF91CF911F9130
:100210000F910895CF93DF93EC010E94CE008823C5
:1002200029F060E070E0CE010E94E400DF91CF9100
:100230000895EF92FF920F931F93CF93DF938C015A
:100240007B01C0E5D3EC03C02097E1F021970E9429
:10025000CE008823C9F3CD2BA9F0E8012196F8013F
:10026000208188819927982F8827B701820F911DB7
:100270000E94E400282F882391F380E090E0213051
:1002800031F403C080E090E002C081E090E0DF91B3
:10029000CF911F910F91FF90EF90089504C082E0DD
:1002A00090E00E940A0180911F018823C1F381E040
:1002B0000E945C0608951F930E944E0163E070E067
:1002C00083E191E00E94810614E60E94CE0088231B
:1002D00069F480E090E00000019629E28432920700
:1002E000D1F7115090F780E090E007C060E070E037
:1002F00083E191E00E94190199271F9108950097C9
:1003000021F077270E9481060895862F99270E9461
:100310005F0608958F929F92AF92BF92CF92DF9225
:10032000EF92FF920F931F93CF93DF93CDB7DEB77A
:1003300022970FB6F894DEBF0FBECDBFC988DA880A
:100340000C898B89E82EFF24AA24BB2445E1842E46
:10035000912C8C0E9D1E9A8289820E944E01B701BB
:10036000C6010E94810607FD25C0002361F110E04F
:1003700006C02050304CC9F01F5F011721F1E98100
:10038000FA81808191813496FA83E983349762817E
:1003900073819B012070307C2115310551F70E943B
:1003A00081061F5F011759F70EC0CB019F730E9492
:1003B0005F06E2CFE981FA813296FA83E983B2904F
:1003C000A2900F77D2CFB501C6010E9419018823F0
:1003D00009F4C1CF22960FB6F894DEBF0FBECDBF91
:1003E000DF91CF911F910F91FF90EF90DF90CF9011
:1003F000BF90AF909F908F9008958FEE90EC9F9359
:100400008F931F921F9289E090E09F938F9380E0DB
:1004100091E09F938F9382E08F9383E08F9386E1A7
:1004200091E09F938F930E948A018DB79EB70C969F
:100430000FB6F8949EBF0FBE8DBF08950E94800333
:100440000E945B01882309F408950E94FD011F9218
:1004500086E08F938DE091E09F938F930E948A01B5
:100460001F9284E08F9389E091E09F938F930E9485
:100470008A010E94EE058DB79EB708960FB6F894D4
:100480009EBF0FBE8DBF089580917C0290917D022A
:10049000089570937D0260937C0290937B02809319
:1004A0007A02089520917A0230917B02280F391F39
:1004B00030937B0220937A020895FF920F931F934B
:1004C000CF93DF93EC018B01F42E80917A0290910F
:1004D0007B02009751F481E090E00E940A01809134
:1004E0007A0290917B020097B1F3019790937B027F
:1004F00080937A0282E00E945C06FF2031F08881BE
:10050000998190620E94740605C0888199819061EA
:100510000E947406C8010E947406DF91CF911F915A
:100520000F91FF900895EF92FF920F931F93CF9337
:10053000DF93EC010E9425067C010E9425068C01B8
:10054000C7019F700E94A103FC010115110501F173
:100550002197229760F0892B51F0C7018070907F1E
:1005600020E18030920739F08050904269F0C80154
:100570000E9432060DC080859185892BC1F31093AE
:10058000DA020093D90204C0B801CF010E942E0AFA
:10059000DF91CF911F910F91FF90EF90089504C0CC
:1005A00080E090E00E940A018091D9029091DA02E5
:1005B0000097B1F301979093DA028093D9020E94D9
:1005C0001D06992708951F93182F11501F3F21F0E2
:1005D0000E94CF021150E0F71F9108951F930E94CF
:1005E000CF02182F0E94CF029927982F8827810FBA
:1005F000911D1F910895EF92FF920F931F93CF9338
:10060000DF93EC01E981FA818081918183529041ED
:1006100019F080E090E052C08881823891F08338F0
:10062000B9F0813819F081E090E048C081E090E0B5
:100630009093850280938402F093F302E093F20298
:100640003DC0109285021092840281E090E036C095
:100650008091820290918302892B29F30680F78191
:10066000E02D00851185C8010E945D497C01A8012B
:10067000BC0189819A810E94360720917E023091C7
:100680007F02A80161E070E0C7010E943549181699
:10069000190644F480917E0290917F020E94DF4708
:1006A000892B39F0109283021092820281E090E04F
:1006B00005C0C7010E945A4981E090E0DF91CF91C7
:1006C0001F910F91FF90EF900895CF93DF93CDB7D7
:1006D000DEB723970FB6F894DEBF0FBECDBF898378
:1006E0007B836A83CE0101960E94FB0299272396A1
:1006F0000FB6F894DEBF0FBECDBFDF91CF91089546
:100700008FEF9FEF9093DE028093DD02089580913A
:10071000DD029091DE028F5F9F4F81F4EDEDF2E0FC
:10072000119282E0E23FF807D9F78FEF9FEF9093A5
:10073000DE028093DD02CF014597089580E090E0CE
:1007400008952091DD023091DE022817390719F44F
:100750008DED92E0089580E090E00895FC0185859C
:100760009685892B19F08FEF90E0089580E090E056
:1007700008950F931F93CF93DF93CDB7DEB72497E0
:100780000FB6F894DEBF0FBECDBF64E070E0CE01BF
:1007900001960E9446068A819B810E94A1038C01DA
:1007A000009759F00E94B007B80185E00E946503E8
:1007B0008FEF9FEFF8019183808324960FB6F89412
:1007C000DEBF0FBECDBFDF91CF911F910F91089576
:1007D000CF93DF93CDB7DEB72B970FB6F894DEBF7C
:1007E0000FBECDBF6BE070E0CE0101960E944606C1
:1007F0008981882301F50E948703BC01892B09F1B7
:100800008A819B81FB0181939193DE0114969E0165
:10081000265F3F4F8D918193A217B307D9F7FB0154
:100820003D96CB01459611928E179F07E1F784E024
:100830000E9465030DC060E070E089E00E946503DE
:1008400007C080E4898360E070E089E00E9465036E
:100850002B960FB6F894DEBF0FBECDBFDF91CF91C0
:100860000895EF92FF921F93CF93DF93CDB7DEB73A
:100870002A970FB6F894DEBF0FBECDBF82E0E82EF8
:10088000F12CEC0EFD1E69E070E0C7010E944606E7
:100890008A81882319F48B81882309F111E00E9451
:1008A0001D06813051F11123B9F48EE0898381E076
:1008B00090E09F938F93CE0101969F938F9386E054
:1008C00090E09F938F93FF92EF9282E08F9383E06B
:1008D0008F9389E191E02DC08DE08983E8CF8C81F1
:1008E0008823E1F68D818823C9F68E818823B1F6AD
:1008F0008F81811181E0182FD2CF0E948703892B2D
:1009000091F2112391F281E0898381E090E09F933D
:100910008F93CE0101969F938F9386E090E09F93F3
:100920008F93FF92EF9282E08F9383E08F938CE11D
:1009300091E09F938F930E948A018DB79EB70C968A
:100940000FB6F8949EBF0FBE8DBF2A960FB6F894CF
:10095000DEBF0FBECDBFDF91CF911F91FF90EF9013
:1009600008950F931F93CF93DF93CDB7DEB72697EC
:100970000FB6F894DEBF0FBECDBF66E070E08E010B
:100980000F5F1F4FC8010E94460686E090E09F93CC
:100990008F931F930F9381E08F9383E08F9380E277
:1009A00091E09F938F930E948A018DB79EB708961E
:1009B0000FB6F8949EBF0FBE8DBF26960FB6F89463
:1009C000DEBF0FBECDBFDF91CF911F910F91089574
:1009D000FF920F931F93CF93DF93CDB7DEB7279787
:1009E0000FB6F894DEBF0FBECDBF84E0F82EF982BB
:1009F0008E010E5F1F4F66E070E0C8010E94460640
:100A00008CE090EC9F938F931F921F9284E090E074
:100A10009F938F9386E291E09F938F9381E090E084
:100A20009F938F93CE0101969F938F9386E090E0E2
:100A30009F938F931F930F93FF9283E08F9383E293
:100A400091E09F938F930E948A018DB79EB7449641
:100A50000FB6F8949EBF0FBE8DBF27960FB6F894C1
:100A6000DEBF0FBECDBFDF91CF911F910F91FF90E1
:100A700008950F931F930E941D06082F882361F08D
:100A800010E082E090E00E9432060E9425060E945B
:100A900052021F5F0117A9F71F910F910895EF925E
:100AA000FF920F931F93CF93DF93EC017B010E9482
:100AB0001D06182F0E941D06082F1F30D1F110317E
:100AC00090F0133109F454C0143108F441C01631C8
:100AD00009F45AC01731F1F58630E1F50E94B104EE
:100AE000C0E0D0E073C0143009F447C01530C8F13D
:100AF000153009F456C01E3069F50E941D0680931A
:100B00001F010E942506C330D10508F04FC021E027
:100B1000C1E0D0E0043008F459C0E114F10419F048
:100B2000213009F44CC0802F992703970E94320688
:100B30004DC00E941D060E941D0680931F010E9449
:100B4000250620E0C817D907E9F0C22FDD273EC0EF
:100B5000103109F1802F99270E943206C0E0D0E0C1
:100B600035C01330B9F70E94E803C0E0D0E02EC0D2
:100B70000E943905C0E0D0E029C00E943104C0E0E5
:100B8000D0E024C021E0E1CF863021F70E94E804C4
:100B9000C0E0D0E01BC099270E943206C2E0D0E03E
:100BA00015C00E94B903C0E0D0E010C020E0C81713
:100BB000D90719F0C22FDD27ADCF21E0FBCF602F81
:100BC000772763507040C7010E944606CE01DF912F
:100BD000CF911F910F91FF90EF900895CF93DF93E6
:100BE000CDB7DEB728970FB6F894DEBF0FBECDBFE6
:100BF000CE0101969F938F9380E88F9383E08F932C
:100C00008AE291E09F938F930E948A016A817B819F
:100C10008D819E810E9449028DB79EB706960FB6C0
:100C2000F8949EBF0FBE8DBF28960FB6F894DEBF16
:100C30000FBECDBFDF91CF9108950E94CE008823D3
:100C4000E1F30E94C600992708951F930E941D0694
:100C5000182F0E941D069927982F8827810F911D14
:100C60001F9108950F931F93CF93DF938C01892BCE
:100C700041F0C0E0D0E00E941D0621960C171D0730
:100C8000D1F7DF91CF911F910F9108950F931F938B
:100C9000CF93DF936115710551F0EC018B01080FC3
:100CA000191F0E941D068993C017D107D1F7DF9144
:100CB000CF911F910F9108950E94BE0008950F9348
:100CC0001F93CF93DF938C01892B49F0C0E0D0E0D4
:100CD00080E00E945C0621960C171D07C9F7DF9182
:100CE000CF911F910F9108950F931F938C010E9434
:100CF0005C06012F1127802F0E945C061F910F9127
:100D000008950F931F93CF93DF936115710551F0F1
:100D1000EC018B01080F191F89910E945C06C01716
:100D2000D107D1F7DF91CF911F910F9108950F93C4
:100D30001F93CF93DF938C01892B51F0C0E0D0E05B
:100D40000E941D060E945C0621960C171D07C1F724
:100D5000DF91CF911F910F910895CF92DF92EF9283
:100D6000FF920F931F93CF93DF936C018A017B0156
:100D70000E9444020497F601C681D7811B870A8727
:100D80001093DC020093DB028017910720F490930C
:100D9000DC028093DB026091DB027091DC026C5F0D
:100DA0007F4F41E0CE010E945D02C8010E9474069F
:100DB000F601828193810E9474066091DB0270913A
:100DC000DC026017710760F031C040E0CE010E9484
:100DD0005D026091DB027091DC026017710730F5F3
:100DE000C7010E9481062091DB023091DC02021BC8
:100DF000130B8A859B85821B930B9B878A87E20E48
:100E0000F31E9093DC028093DB020E944402609107
:100E1000DB027091DC0286179707B8F60E94440245
:100E2000BC019093DC028093DB02CFCF011511054A
:100E3000A1F0B801C7010E9481068A859B85801BAD
:100E4000910B9B878A878091DB029091DC02801B4B
:100E5000910B9093DC028093DB02DF91CF911F9185
:100E60000F91FF90EF90DF90CF900895CF92DF9297
:100E7000EF92FF920F931F93CF93DF93EB01FC014F
:100E8000C680D780F601E084F1844E155F0508F432
:100E90007A01E114F10429F43EC080E090E00E9460
:100EA0000A012091D9023091DA0221153105A9F306
:100EB000F601808591852817390708F4C901AC012E
:100EC000E816F90608F4A701E41AF50A241B350B05
:100ED0003093DA022093D902F60180859185841B34
:100EE000950B91878087209781F04115510549F036
:100EF0008A010C0F1D1F0E941D068993C017D10780
:100F0000D1F7E114F10469F606C0CA010E94320665
:100F1000E114F10431F6DF91CF911F910F91FF9011
:100F2000EF90DF90CF900895CF93DF93CDB7DEB7EA
:100F300021970FB6F894DEBF0FBECDBF41E050E061
:100F4000BE016F5F7F4F0E943607898199272196E6
:100F50000FB6F894DEBF0FBECDBFDF91CF910895DD
:100F6000CF93DF93EC018D859E85892B31F0BE01F7
:100F7000635F7F4F82E80E9465031E861D86DF91B6
:100F8000CF910895EF92FF920F931F93CF93DF932A
:100F90007C01062FEA010E94EE02182F10540E94D5
:100FA000EE020E94EE02C730D10520F5612F7727AF
:100FB000202F3327660F771F660F771F660F771F67
:100FC000FB01EE0DFF1D8189928928173907C1F4B5
:100FD000858596859C013F7B368725878070907834
:100FE000892B71F4635F7F4F6E0D7F1D81E80E9436
:100FF000650306C09E012650822F0E94E302D6CFD1
:10100000DF91CF911F910F91FF90EF900895DF92A4
:10101000EF92FF920F931F93CF93DF93EC01F62E85
:10102000E42ED22EB801685F7F4F41E00E945D023E
:10103000C80104960E94740681E090E00E94740644
:101040008F2D0E945C06EE20D1F48C858F5F8C87FB
:10105000882391F08C850E945C06ED2DFF27EE0F12
:10106000FF1FEE0FFF1FEE0FFF1FEC0FFD1F8C8504
:101070009927928B818B06C081E08C87EBCF8E2DD8
:101080000E945C06C8010E947406DF91CF911F91F7
:101090000F91FF90EF90DF9008955F926F927F9293
:1010A0008F929F92AF92BF92CF92DF92EF92FF9278
:1010B0000F931F93CF93DF93CDB7DEB74C01562E1E
:1010C0006A016DB67EB68DB79EB7841B950B0FB6C1
:1010D000F8949EBF0FBE8DBFADB6BEB60894A11CDE
:1010E000B11C452B69F000E010E075010E94CF02B1
:1010F000F70181937F010F5F1F4FC016D106B1F733
:10110000860120E0452D69E0C4010E940708B60170
:10111000C5010E9481060FB6F8947EBE0FBE6DBE5B
:10112000DF91CF911F910F91FF90EF90DF90CF90C3
:10113000BF90AF909F908F907F906F905F90089539
:10114000BF92CF92DF92EF92FF920F931F936C01A9
:10115000B62E0E94EE0230ECE32EE80E0E94EE0264
:1011600004E010E020E04B2D67E0C6010E94070874
:10117000FF24C701805C9F4F0E947406EE0CFF1C89
:10118000EE0CFF1CEE0CFF1C87010C0D1D1DF80161
:10119000878590890E9474068DE090E0E80EF91E24
:1011A000EC0CFD1CB70182E80E946503F80116866D
:1011B00015861F910F91FF90EF90DF90CF90BF9019
:1011C00008952F923F924F925F926F927F928F92EB
:1011D0009F92AF92BF92CF92DF92EF92FF920F93C6
:1011E0001F93CF93DF93CDB7DEB74C01C62E7A01A4
:1011F0002DB63EB68CEF9FEFE80EF91EEDB7FEB7A9
:10120000EE19FF090FB6F894FEBF0FBEEDBFADB6E5
:10121000BEB60894A11CB11C0E94EE0250EC652ED3
:101220005FEF752E680E791E0E94EE022C01E1140C
:10123000F10479F0DD2400E010E00E94CF020A0DF5
:101240001B1DF8018083D3940D2D11270E151F054A
:10125000A0F306E010E020E04C2D65E0C4010E9400
:1012600007087301EE0CFF1CEE0CFF1CEE0CFF1CBC
:101270008701080D191DF801878590890E94740661
:1012800080E090E00E947406C2010E947406F8019A
:1012900025853685C9019F779687858736FD0AC0E3
:1012A0008DE090E0E80EF91EE80CF91CB70181E82A
:1012B0000E9465030FB6F8943EBE0FBE2DBEDF91AF
:1012C000CF911F910F91FF90EF90DF90CF90BF9043
:1012D000AF909F908F907F906F905F904F903F90D6
:1012E0002F900895DF92EF92FF920F931F937C014E
:1012F000D62E04E010E0262F40E064E00E940708AC
:10130000ED2DFF27EE0FFF1FEE0FFF1FEE0FFF1F4C
:10131000EE0DFF1D878590890E94740680E090E0A5
:101320000E9474061F910F91FF90EF90DF90089537
:101330008F929F92AF92BF92CF92DF92EF92FF92E5
:101340000F931F93CF93DF936C01962E0E94AE03F1
:10135000882E8FEF881609F457C0E82CFF240E94CE
:10136000EE025701AA0CBB1CAA0CBB1CAA0CBB1C8E
:10137000E501CC0DDD1D906C9E878D870E94EE02ED
:10138000988B8F87DC8ACB8A08E010E020E0492D1B
:1013900063E0C6010E940708C701805C9F4F0E945E
:1013A00074068F8598890E9474060D851E85C80174
:1013B0009F739E878D87B501635F7F4F6C0D7D1D89
:1013C00080E80E9465038823C1F080E090E00E94DD
:1013D00074061E870D8780E090E00E947406AC0CB6
:1013E000BD1CF50185859685892B59F19394492D6E
:1013F000682DC6010E94720924C082E090E00E941C
:1014000074061E861D86E7CF0E94EE020E94EE0241
:101410007C0108E010E020E0492D63E0C6010E9455
:10142000070880E090E00E947406C7010E947406DD
:1014300084E090E00E94740678EFA72E77E0B72E44
:10144000CACFDF91CF911F910F91FF90EF90DF9066
:10145000CF90BF90AF909F908F900895EF92FF92A2
:101460000F931F93CF93DF938C017093DA026093F5
:10147000D9020E94EE02F801918780870E94EE0255
:1014800081309105E1F0EC01CC0FDD1FCC0FDD1FA9
:10149000CC0FDD1FC00FD11FC35FD140BE0183E859
:1014A0000E946503F801408551854115510509F4F5
:1014B00047C060E070E0CE010E94360741C00E9444
:1014C000CF02F82E0E94CF02E82E0E94EE02AC015D
:1014D000F8012085318504968217930721F0822F29
:1014E0000E94E3022DC0F5E0FF1609F1FF1558F048
:1014F00082E0F81691F0E4E0FE1659F46E2DC80172
:101500000E94E1081DC0F6E0FF1661F088E0F816C1
:1015100099F0842F0E94E30213C06E2DC8010E942F
:1015200098090EC06E2DC8010E94A00809C06E2D3A
:10153000C8010E94C20704C06E2DC8010E944D0858
:10154000DF91CF911F910F91FF90EF90089504C00C
:1015500080E090E00E940A018091820290918302D3
:10156000892BB1F708958091820290918302892B93
:1015700041F40E947E0E8091820290918302892B19
:10158000C1F380E40E94F60D0E94A70A80E80E9441
:10159000F60DEFCFCF93DF9380E890E00E945D4996
:1015A000EC018091820290918302892B69F1209154
:1015B0007E0230917F0240E850E061E070E0CE01B1
:1015C0000E94B348AC0118161906D4F48091840225
:1015D00090918502892B29F3BE018091F2029091AE
:1015E000F3020E94AD0680918002909181020E94D8
:1015F000DF478091820290918302892BC1F604C05B
:101600001092830210928202CE010E945A49DF9109
:10161000CF9108958F929F92AF92BF92CF92DF9217
:10162000EF92FF920F931F93CF93DF93CDB7DEB767
:101630002F970FB6F894DEBF0FBECDBF80E092ECBF
:10164000A1E0B0E08D839E83AF83B88719821A82B0
:101650001B821C8240E060E070E08DE791E00E9418
:10166000AF1245E060E073E889EF91E00E94AF12AD
:101670006DE271E081E391E00E9420489093810245
:10168000809380020E94F047AE014B5F5F4F61E0A4
:1016900071E00E94334780918002909181020E9404
:1016A000F047AE014F5F5F4F6BE071E00E94334740
:1016B0000E941E0299E0892E912C8C0E9D1EF40131
:1016C000ACE5B1E087E00D9001928150E1F787E34E
:1016D00091E00E94312E5B016C0185E491E00E9453
:1016E000312E7B018C01A6019501B40183E591E0C7
:1016F0000E942D3120E030E140E050E063EB7AE0E1
:1017000088E591E00E9459131092830210928202A0
:1017100081E0E82EF12C0E94082B8C0167E170E03B
:101720000E94AB2B6DE271E0C8010E948647909346
:101730007F0280937E02F0928302E09282020E94F6
:10174000CA0A80917E0290917F020E9446471092C1
:101750007F0210927E02C8010E94562ADCCF80933D
:10176000760108950E941A1120E033E040E050E035
:101770006AE07BE081E791E00E9459138EEF0E94BE
:10178000F60D0E947E0E0E94B50D209176012F3F2E
:10179000C1F395B785B7837E822B85BF85B78062FD
:1017A00085BF889585B78F7D85BF85B7837E9C7102
:1017B000892B85BF0E947E0E0E94B50D2091760177
:1017C0002F3F39F7DECF0F931F93CF93DF93009115
:1017D0008702109188028017910708F062C0AC015F
:1017E0004A5F5F4F4430510508F458C0E09134031C
:1017F000F0913503309709F454C064E373E0C0E01E
:10180000D0E0A0E0B0E004C0BF016E5F7F4FFC01FC
:10181000208131812417350768F04217530709F4F6
:1018200048C0209729F0888199812817390710F43A
:10183000EF01DB0182819381009731F7CE01209780
:10184000D9F128813981CA010A968217930760F578
:10185000FA01EC0FFD1F241B350B318320838A8195
:101860009B81938382839A0159834883ED93FC93F0
:10187000021B130B10938802009387022C0F3D1F4D
:10188000245030408FEE9EEBADEABEEDF90180832F
:101890009183A283B383CE0102960EC044E050E050
:1018A000A5CF80E090E008C08A819B818D939C93B6
:1018B000DFCFEF01DB01C5CFDF91CF911F910F91FA
:1018C0000895CF93DF93DC0112974D915C911197AE
:1018D000E0913403F0913503C4E3D3E0309759F13C
:1018E00020813181CF01820F931F8A179B07A1F4BA
:1018F00034C0A817B90708F449C0EF012296028046
:10190000F381E02D3097B9F020813181C9018E0F2C
:101910009F1F8A179B0709F1AE17BF0750F7B983BE
:10192000A883CA018A0F9B1F8E179F0791F1ED01B3
:10193000FB83EA8305C0FD0113821282B983A88369
:101940008091870290918802840F951F909388025E
:101950008093870280E090E027C0240F351F3183F9
:10196000208382819381D901AE0FBF1FA817B907C9
:1019700039F78D919C911197280F391F318320835E
:10198000ED018A819B8193838283DACF8FEF9FEF72
:101990000BC0240F351F11963C932E9382819381A7
:1019A000FD0193838283CCCFDF91CF910895FC0119
:1019B00061937193CF010E94610C08958091870219
:1019C0009091880208950F931F93CF93DF938C011A
:1019D0000E94E30BEC01009729F0A80160E070E0A1
:1019E0000E941F4ACE01DF91CF911F910F91089560
:1019F000CF93DF93DC019B01EC01788F6F8B1D820D
:101A00001C820FB6F8940F92EB01E881F9818FEFF9
:101A1000EF3FF80769F1309791F00F900FBEED019D
:101A20009A898289981740F09F012E5F3F4F02806C
:101A3000F381E02D3097A9F70FB6F8940F92ED01DE
:101A4000FB83EA83F901B183A083EA81FB813097AC
:101A5000C1F084819581892BA1F08C819D812481A5
:101A60003581820F931F9D838C831582148209C058
:101A7000ED018C819D8101969D838C83E0E0F0E0F7
:101A8000DECF0F900FBEDF91CF910895CF93DF93FC
:101A9000DC01EB010FB6F8940F92E881F9810F9009
:101AA0000FBE8FEFEF3FF80789F1309779F1EA1712
:101AB000FB0721F40BC0AE17BF0741F0EF012296E0
:101AC0000280F381E02D3097B1F720C00FB6F89473
:101AD0000F92FD018281938199838883848195810E
:101AE000892B69F00280F381E02D309729F0ED0118
:101AF0008C819D8195838483FD01158214820F90D2
:101B00000FBEED011B821A82188E1F8ADF91CF91C2
:101B10000895FB01168A158A82E0878768E373E0DF
:101B2000CF010E94F80C08950F931F93CF93DF937A
:101B30008C01C0913603D0913703209731F40EC049
:101B40000990D881C02D209749F0B801CE010696A2
:101B50000E94264A892BA1F7CE0102C080E090E0C6
:101B6000DF91CF911F910F910895E0913C03F09187
:101B70003D03309741F0838994890E94610C109253
:101B80003D0310923C030895CF93DF93C091360339
:101B9000D09137030E94B50D2097E9F080913A0368
:101BA00090913B03C817D90721F40AC0C817D90779
:101BB00049F0FE010990D881C02D2097B9F70FC0D8
:101BC000E6E3F3E0888199819183808380913A03F1
:101BD00090913B0304C080913A0390913B03909312
:101BE0003D0380933C03DF91CF9108950F931F93A2
:101BF000182FE0913A03F0913B03028968E373E008
:101C0000CF010E94460DE0913A03F0913B03128B05
:101C10001F3F01F168E373E080913A0390913B0329
:101C20000E94F80CE0913A03F0913B038091380355
:101C300090913903E817F90751F082E087870FB6D2
:101C4000F8940F920E941A130F900FBE06C081E005
:101C5000878703C00E94C40DE5CF802F99271F916D
:101C60000F9108958FEF0E94F60D0895CF93DF93A3
:101C7000C0913603D0913703209711F10FB6F89435
:101C80000F928C819D810F900FBE892BA1F0EF895F
:101C9000F88D0FB6F8940F928C819D8101979D83EA
:101CA0008C830F900FBE808191818F5F9F4F19F0C1
:101CB000CF010E9422110990D881C02D2097F1F602
:101CC0000E94C80FE0913A03F0913B0380913803E2
:101CD00090913903E817F90771F08785813041F059
:101CE0000FB6F8940F920E941A130F900FBE03C004
:101CF00082E08787F5CFDF91CF910895E0913A0395
:101D0000F0913B0382819381892B69F068E373E052
:101D1000CF010E94460D68E373E080913A039091F1
:101D20003B030E94F80C0E94360E089580914003F8
:101D300090914103A0914203B09143030196A11DEC
:101D4000B11D8093400390934103A0934203B0934D
:101D500043030895CF93DF93EC011B821A82E09135
:101D60003E03F0913F03309751F1288539854A852C
:101D70005B8580859185A285B385281739074A0739
:101D80005B0760F425C09C01AD0180859185A2852B
:101D9000B385281739074A075B07D0F0281B390B92
:101DA0004A0B5B0BDA01C901288739874A875B87B1
:101DB000FB83EA830190F081E02D309721F71982AF
:101DC0001882EA81FB81309799F0D183C08314C0D7
:101DD000821B930BA40BB50B80879187A287B387D7
:101DE000F983E883D383C283EA81FB81309769F763
:101DF000D0933F03C0933E03DF91CF9108950FB678
:101E0000F8940F92609140037091410380914203D6
:101E1000909143030F900FBE08952F923F924F92DF
:101E20005F926F927F928F929F92AF92BF92CF926A
:101E3000DF92EF92FF920F931F93CF93DF93CDB773
:101E4000DEB724970FB6F894DEBF0FBECDBF0E9459
:101E5000FF0E5B016C010E9415149B01AC01C601D1
:101E6000B5010E946F4A39014A010E9415141B01F5
:101E70002C010E94151469837A838B839C83C4018F
:101E8000B30128EE33E040E050E00E94304A7B018D
:101E90008C01C401B301A20191010E94304AA61A2B
:101EA000B70AC80AD90AC601B50128EE33E040E0F6
:101EB00050E00E94304A29813A814B815C810E9426
:101EC0006F4AE20EF31E041F151FC801B7012496C6
:101ED0000FB6F894DEBF0FBECDBFDF91CF911F913B
:101EE0000F91FF90EF90DF90CF90BF90AF909F90B9
:101EF0008F907F906F905F904F903F902F900895BC
:101F0000EF92FF920F931F930E94FF0E7B018C01B3
:101F10000E9415149B01AC01C801B7010E946F4AD1
:101F2000CA01B9011F910F91FF90EF900895CF93CF
:101F3000DF93FC01A281B3811097E9F08081918148
:101F40008D939C93C081D1812097E1F08281938110
:101F50009B838A8388859985AA85BB852085318561
:101F600042855385820F931FA41FB51F88879987C9
:101F7000AA87BB8707C08081918190933F0380939C
:101F80003E03E0CFCF010E94610CDF91CF91089515
:101F9000CF92DF92EF92FF920F931F93CF93DF9335
:101FA0000E94FF0E2091890230918A0240918B029B
:101FB00050918C027B018C01E21AF30A040B150B81
:101FC0006093890270938A0280938B0290938C02B3
:101FD000C0913E03D0913F036E01209709F460C089
:101FE000E114F1040105110509F45AC088859985A9
:101FF000AA85BB85E816F9060A071B0798F48E190F
:102000009F09A00BB10B88879987AA87BB87009788
:10201000A105B105C9F1EE24FF2487016E012097C7
:10202000F9F63EC0E81AF90A0A0B1B0B1886198646
:102030001A861B86EC85FD85309721F06E857F859D
:10204000CE0109958C819D81AE81BF81888799875A
:10205000AA87BB870097A105B105D1F0E0913E03A7
:10206000F0913F03C081D181D0933F03C0933E03E1
:10207000209711F01B821A82C6010E94AA0EC091FD
:102080003E03D0913F03A8CFEE24FF248701D2CF97
:10209000CE010E94970FC0913E03D0913F039CCF89
:1020A000DF91CF911F910F91FF90EF90DF90CF9034
:1020B00008958F929F92AF92BF92CF92DF92EF924C
:1020C000FF920F93CF93DF936B017C015A0149017B
:1020D00080E190E00E94E30BEC01892B31F10E943A
:1020E000FF0E6C0D7D1D8E1D9F1D2091890230916C
:1020F0008A0240918B0250918C02621B730B840BFD
:10210000950B688779878A879B8700FF09C01C82A7
:102110001D821E821F82BD86AC869F868E8605C06C
:10212000CC82DD82EE82FF82F6CFCE01DF91CF91AD
:102130000F91FF90EF90DF90CF90BF90AF909F9066
:102140008F9008950F93CF93DF930E945910EC0165
:10215000009711F00E94AA0ECE01DF91CF910F914E
:102160000895CF92DF92EF92FF920F936A01790167
:102170000E941A149701A6010E94A2100F91FF90CD
:10218000EF90DF90CF900895AF92BF92CF92DF9201
:10219000EF92FF920F93CF93DF935B016C01611578
:1021A00071058105910519F1C8E3D3E0BE01809165
:1021B0003A0390913B030E94460DE0913A03F0915F
:1021C0003B0383E08787E0903A03F0903B0301E014
:1021D000970149E85DE0C601B5010E94B110F70121
:1021E000968B858B892B31F00E94360E19C00E9488
:1021F0007E0E16C0E0913A03F0913B03D08FC78B5F
:1022000080913803909139039383828381E087879B
:1022100080913A0390913B03909339038093380364
:10222000DF91CF910F91FF90EF90DF90CF90BF9013
:10223000AF90089586E99EE00E943F1487B78260C0
:1022400087BF0895CF93DF93DC010FB6F8940F9208
:10225000CD91DC9111970F900FBE8FEFCF3FD80734
:1022600009F434C0209741F10FB6F8940F92EA8137
:10227000FB811196FC93EE938C819D81892B41F01B
:10228000309739F18C819D81958384831D821C82D6
:102290000F900FBE8D899E89009721F00E94970FA5
:1022A0001E8A1D8A82E08F8768E373E0CE010E9458
:1022B000F80C81E090E013C00FB6F8940F928FEF06
:1022C0009FEF11969C938E930F900FBE80E090E04D
:1022D00006C08FEF9FEF11969C938E93D7CFDF911F
:1022E000CF9108950F931F93CF93DF93EC010FB617
:1022F000F8940F92888199810F900FBE2FEF8F3F36
:102300009207A9F0892BE9F000E010E0CE010E94CD
:102310002211080F191F0FB6F8940F928881998126
:102320000F900FBE01978E5F9F4F80F30CC00FB6CA
:10233000F8940F92198218820F900FBE00E010E0FF
:1023400002C000E010E0C801DF91CF911F910F9112
:1023500008950F931F930E9472118C010E947E0EAC
:10236000C8011F910F9108950F931F930E9422118E
:102370008C010E947E0EC8011F910F910895CF938A
:10238000DF939C01FB010FB6F8940F92C081D181BD
:102390000F900FBE8FEFCF3FD80709F43FC02097B3
:1023A00009F43CC08D899E892817390731F40DC086
:1023B0008D899E898217930741F0FE0132960A802B
:1023C000DB81C02D2097A1F729C00FB6F8940F929A
:1023D0008A819B81918380838C819D81892B59F097
:1023E000AA81BB811097A9F08C819D81FD01958305
:1023F00084831D821C820F900FBE82E08F8768E36A
:1024000073E0CE010E94F80C8FEF9FEF9E8B8D8BB7
:1024100005C08FEF9FEF91838083EBCFDF91CF914A
:102420000895AF92BF92CF92DF92EF92FF920F93F7
:10243000CF93DF93EC015A016B010FB6F8940F9222
:10244000888199810F900FBE8F5F9F4F09F43EC026
:1024500068E373E080913A0390913B030E94460D3C
:10246000BE0180913A0390913B030E94F80CE091E9
:102470003A03F0913B0383E08787A114B104C104C0
:10248000D104A1F4E0913A03F0913B03168A158A36
:102490000E94360EE0913A03F0913B0385899689BC
:1024A0008F5F9F4FF9F080E090E020C0E0903A030A
:1024B000F0903B0301E09E014FEB51E1C601B501F5
:1024C0000E94B110F701968B858BE2CF0FB6F8947E
:1024D0000F92198218820F900FBE0E947E0E80E02C
:1024E00090E004C0168A158A8FEF9FEFDF91CF919D
:1024F0000F91FF90EF90DF90CF90BF90AF90089535
:10250000FC010FB6F8940F92808191818F5F9F4FED
:1025100011F4118210820F900FBECF010E94111290
:1025200008950F931F93CF93DF938C01C0918D0279
:10253000D0918E02209731F40CC00990D881C02D23
:10254000209739F0B801CE0102960E94264A892BC5
:10255000A1F7CE01DF91CF911F910F910895CF93F5
:10256000DF93EC01892B19F48FEF9FEF23C06115E6
:10257000710511F07D876C8741114E87CE0102965F
:102580000E949112892B81F7EB89FC89309769F4BD
:1025900080918D0290918E0299838883D0938E02D0
:1025A000C0938D0280E090E005C0CE010995892B93
:1025B00079F3DACFDF91CF91089583E180934403DB
:1025C0008FE48093450383E58093460343E150E025
:1025D00064E473E080E090E00E94F825892B19F410
:1025E00080E090E008958FEF9FEF089543E150E081
:1025F00064E473E080E090E00E94FB25892B41F4C5
:1026000080914403833121F4809145038F3419F084
:102610008FEF9FEF0895809146038335C9F780E0DF
:1026200090E008959F918F910F900BBE0F900FBE79
:102630001F9018952F923F924F925F926F927F92C8
:102640008F929F92AF92BF92CF92DF92EF92FF92C2
:102650000F931F93CF93DF938DB79EB7E0913A030B
:10266000F0913B03918B808BE0913803F09139031B
:10267000F0933B03E0933A0381E08787E0913A03CC
:10268000F0913B03808991898DBF9EBFDF91CF91EF
:102690001F910F91FF90EF90DF90CF90BF90AF9080
:1026A0009F908F907F906F905F904F903F902F9072
:1026B0000895AF92BF92CF92DF92EF92FF920F9365
:1026C0001F93CF93DF937C016B015A018901C901EC
:1026D00049960E94E30BEC01009709F472C0080FC1
:1026E000191F980127503040A8014B515040D80184
:1026F0001696F70188E001900D928150E1F7F801FC
:10270000168641505040518B408B4F5F5F4FD48BAA
:10271000C38B8FEE9EEBADEABEED88839983AA83CF
:10272000BB838C839D83AE83BF8388879987AA8769
:10273000BB878C879D87AE87BF8780E4828B8D2D7A
:102740009927F9018583C68280E8838312821482E7
:10275000A1828B2D9927808322E133E1832F992752
:10276000FA01828B238B8091360390913703F80115
:1027700091838083109337030093360382E0F82E11
:10278000F786168A158A108E178A68E373E0C801E7
:102790000E94F80CE0913A03F0913B033097A1F0CE
:1027A0008091380390913903E817F90741F0F786D3
:1027B0000FB6F8940F920E941A130F900FBEC80123
:1027C00008C080E090E005C00FB6F8940F924CCF9F
:1027D000E7CFDF91CF911F910F91FF90EF90DF90A6
:1027E000CF90BF90AF9008951F93182F60918F02E4
:1027F00070919002809191029091920220EA3FE0C4
:1028000040E050E00E946F4A822F932F0197F1F72A
:102810001A95D1F71F91089560918F0270919002DF
:102820008091910290919202089560E074E080E0BE
:1028300090E00895AF92BF92CF92DF92EF92FF9215
:102840000F931F937B018C010E9415145B016C0197
:10285000C801B70128EE33E040E050E00E94304A62
:10286000A60195010E946F4ACA01B9011F910F91FB
:10287000FF90EF90DF90CF90BF90AF900895BC0194
:1028800087B78D7F87BF80B7886080BF12BE82E028
:1028900083BF80B7992787709070892BD1F781E02B
:1028A00086BF0FB6F8940F9281E090E0A0E0B0E010
:1028B000B6B7B170E9F3B6BF0894811D911DA11D93
:1028C000B6B7B170C9F3BB270F900FBE880F991F21
:1028D000AA1FBB1F880F991FAA1FBB1F880F991F14
:1028E000AA1FBB1F880F991FAA1FBB1F880F991F04
:1028F000AA1FBB1F880F991FAA1FBB1F880F991FF4
:10290000AA1FBB1F80938F0290939002A093910205
:10291000B093920287B78D7F87BF80B7886080BFF2
:1029200012BE89E083BF8FE181BF80B7992787708E
:102930009070892BD1F782E086BF40E050E087E7B6
:1029400091E00E94101E08959C01FB0187B7482F5B
:1029500055274270507087B78D7F87BF2031310572
:10296000D1F02131310564F02231310509F12231F4
:1029700031056CF520E030E087B7826087BF31C059
:1029800021153105C1F021303105B9F02FEF3FEFAE
:10299000452B91F726C006B601FC14C011821082A7
:1029A000452B31F080819181806891838083E2CFD3
:1029B00020E030E016C040E050E082E086BF20E03A
:1029C00030E0E6CF81E090E091838083E9CF203250
:1029D0003105E1F68EE090E09183808320E030E0E5
:1029E000D7CFC90108951F920F920FB60F921124ED
:1029F0002F933F934F935F936F937F938F939F9307
:102A0000AF93BF93EF93FF9387E791E00E94021E7D
:102A1000FF91EF91BF91AF919F918F917F916F91B6
:102A20005F914F913F912F910F900FBE0F901F908C
:102A30001895FC01A281B38140919402242F332781
:102A4000C90180739070892B69F024FF2FC083E146
:102A50008CB9406440939402809194028F7C80935F
:102A60009402089547FD3FC082859385892B49F1E3
:102A70008285938501979387828780919502882329
:102A800009F442C0509A8D918CB99D01868197813D
:102A9000A817B90709F43FC0338322832285338501
:102AA000848595852817390701F1089581E18CB94E
:102AB0004F7B40939402809194028F7C8093940288
:102AC0000895559813861286A089B1891097F1F060
:102AD000FFEFAF3FBF0749F3FD0184819581019668
:102AE00095838483089555980895A089B189109796
:102AF00069F08FEFAF3FB807C1F2FD018481958186
:102B000001969583848308955098BDCF8FEF9FEFF2
:102B1000918B808B089524813581BECF1F93CF93F5
:102B2000DF93DC014BB180919302482B40939302D9
:102B30001CB150919402552321F0133151F1113100
:102B4000F1F1ED012A853B8588859985281739079C
:102B5000E0F4B9016F5F7F4F61307105A9F1552332
:102B6000E9F4ED91FC91119711931196FC93EE937A
:102B70002D913C911197FD01868197812817390786
:102B800091F1ED017B876A873DC0486040939302D5
:102B900039C0559850685093940234C0ED018E8529
:102BA0009F8568177907E8F256FDDBCF5D9B26C04D
:102BB00083E18CB950645F7D50939402D2CF559AD3
:102BC0005F77509394021EC0ED01E889F989309730
:102BD00081F08FEFEF3FF80721F284819581019614
:102BE00095838483BECF8481958111969C938E9327
:102BF000C8CF8FEF9FEF998B888BB3CF50625093E4
:102C00009402AFCFDF91CF911F9108950FB6F89442
:102C10000F9288EB8AB90F900FBE0895529912C097
:102C20008091950082FD07C08091950081FF10C0C2
:102C300086E090E008958091950081FF06C088E0CD
:102C400090E0089589E090E0089587E090E008958D
:102C500085E090E008958091950085FF0AC08091FD
:102C6000950084FF03C081E090E0089582E090E049
:102C7000089580E090E008958091950083FF03C05F
:102C800082E090E0089581E090E0089580919302C1
:102C9000682F7727CB01929582958F7089279F7037
:102CA00089279C014427552721703070407050704F
:102CB00063FD226062FD246080919402882321F0EC
:102CC00086FD18C087FD19C041FF416043FF446085
:102CD00080919502882339F0CA01B9018064589B1C
:102CE00007C080610895CA01B90180685899F9CF79
:102CF00080620895426087FFE7CF4860E5CFEF929A
:102D0000FF920F931F937B018C0180919402882383
:102D100089F00FB6F8940F9200FF39C08F7B809333
:102D2000940202FF3BC0809194028F7780939402BB
:102D30000F900FBE06FF03C081E08093950207FF4E
:102D400002C01092950204FD589A05FD5898E0FEC5
:102D500005C0809193028F7E80939302E1FE05C0AF
:102D600080919302877F80939302E2FE05C0809159
:102D700093028B7F809393020E944616687FE6162B
:102D8000F7060807190791F480E090E011C001FFF1
:102D9000C8CF80648093940202FDC5CF03FFC8CFE3
:102DA00080919402806880939402C2CF8FEF9FEF4E
:102DB0001F910F91FF90EF9008958091950086FFED
:102DC0000AC0129B0DC093E08091950080FD946035
:102DD000892F99270895599B05C080E290E00895B6
:102DE00091E0F2CF80E090E00895809194028823F2
:102DF00029F060E270E080E090E0089560E070E02B
:102E000080E090E00895EF92FF920F931F937B0173
:102E10008C0165FF0EC080919402882391F00E947E
:102E2000F516E616F70608071907A1F480E090E00A
:102E300013C00FB6F8940F92109294020F900FBE29
:102E4000EECF0FB6F8940F9281E4809394020F9026
:102E50000FBEE5CF8FEF9FEF1F910F91FF90EF9087
:102E60000895559A089590919402992399F096FFA8
:102E700011C00FB6F8940F925D9B0DC081E18CB923
:102E80009F7E90939402809194028F798093940214
:102E90000F900FBE0895906190939402F4CF0FB6F7
:102EA000F8940F925798569855980F900FBE8AE055
:102EB0000E94F4135498539808951F93182F0E945A
:102EC0004F17812F992780FF0DC081FF23C0129AD1
:102ED00082FF23C08091950081608093950059986E
:102EE0005E9A0DC085FF14C0599A809195008E7F1F
:102EF00080939500809195008F7B809395000E9430
:102F000006160E94DD16181771F480E090E00DC0DF
:102F10005998EBCF129882FDDDCF809195008E7F7E
:102F200080939500DCCF8FEF9FEF1F9108951F9343
:102F3000182F0E944F17113059F0123079F00E946B
:102F400006160E943C16181779F480E090E00EC037
:102F500080919500877F80939500F1CF80919500B7
:102F6000886080939500EBCF8FEF9FEF1F910895BE
:102F70001F93182F0E944F171130C1F0113058F0D5
:102F80001230F9F00E9406160E942B16181721F530
:102F900080E090E023C0809195008F7E8093950023
:102FA000809195008F7D80939500ECCF8091950066
:102FB0008061809395008091950080628093950058
:102FC000E1CF809195008F7E809395008091950050
:102FD000806280939500D6CF8FEF9FEF1F91089569
:102FE0001F93182F0E944F175298809195008D7F44
:102FF00080939500809195008B7F8093950017308A
:10300000B9F0183058F41630C9F00E9406160E9424
:103010000E161817C9F480E090E018C0183019F0A7
:10302000193099F7529A80919500826080939500AB
:1030300080919500846080939500E7CF8091950002
:10304000826080939500E1CF8FEF9FEF1F910895ED
:10305000EF92FF920F931F937B018C010E944F17F9
:103060008091950086FD17C059990DC0EE0CFF1C8C
:10307000001F111FEE0CFF1C001F111FEE0CFF1C88
:10308000001F111F08C0EE0CFF1C001F111FEE0CCB
:10309000FF1C001F111F0E940C14A80197010E9421
:1030A0006F4A2F5F3F4F4F4F5F4F5695479537956C
:1030B00027952150304029B9232F332720939000A2
:1030C0000E94061680E090E01F910F91FF90EF9014
:1030D00008958F929F92AF92BF92CF92DF92EF921C
:1030E000FF920F931F9389B090909000809195006C
:1030F00086FD0EC0599B06C018E0A12EB12CC12C34
:10310000D12C0BC0B0E1AB2EB12CC12CD12C05C001
:1031100002E0A02EB12CC12CD12C0E940C147B01FA
:103120008C01282D3327892D9927982F8827282B24
:10313000392B442755272F5F3F4F4F4F5F4FC60115
:10314000B5010E94304A9B01AC01C801B7010E9441
:103150006F4ACA01B9011F910F91FF90EF90DF9064
:10316000CF90BF90AF909F908F90089540E050E037
:1031700060E070E08BE392E00E94101E40E050E0BF
:1031800060E070E081E492E00E94101E80E090E038
:10319000089542EC51E06EE875E18BE392E00E9405
:1031A000101E892B19F08FEF9FEF089540EB51E02F
:1031B00069E175E181E492E00E94101E892B19F407
:1031C00080E090E0089540E050E060E070E08BE344
:1031D00092E00E94101E8FEF9FEF08959C01FB016B
:1031E0008AB1482F552740785070579820313105C3
:1031F000C1F02131310554F022313105C1F02231C5
:1032000031052CF580E090E0579A0895211531059D
:1032100089F02130310581F08FEF9FEF452BA1F729
:1032200008955F991EC011821082452B51F480E0F1
:1032300090E0089540E050E08CB18CB180E090E0E7
:10324000EDCF80819181806891838083DBCF2032B4
:10325000310511F780E190E09183808380E090E078
:10326000DDCF81E090E091838083DFCF1F920F92CA
:103270000FB60F9211242F933F934F935F936F9349
:103280007F938F939F93AF93BF93EF93FF938BE3C2
:1032900092E00E94021EFF91EF91BF91AF919F912A
:1032A0008F917F916F915F914F913F912F910F90EF
:1032B0000FBE0F901F9018959C01FB018AB1482FFB
:1032C00055274072507055982131310511F1223146
:1032D000310564F02231310501F12032310501F16F
:1032E0008FEF9FEF452BD9F0559A089521153105A1
:1032F000A1F020313105A1F75D9B19C081E090E07C
:1033000091838083452B49F08081918180689183EE
:10331000808380E090E0559A089580E090E00895E1
:1033200080E190E09183808380E090E0DBCF1182A8
:103330001082E8CF1F920F920FB60F9211242F9395
:103340003F934F935F936F937F938F939F93AF932D
:10335000BF93EF93FF9381E492E00E94021EFF91DE
:10336000EF91BF91AF919F918F917F916F915F91FD
:103370004F913F912F910F900FBE0F901F90189576
:1033800082E28093008390E003C09F5F953121F03B
:103390008091078386FFF9CF80E4809307830895A7
:1033A000FC016115710569F09B0121503040832FAC
:1033B0009927982F8191809310832150D8F79150AD
:1033C000C8F70895CF93DF93FC01C189D2898A851C
:1033D0009B85AC85BD850196A11DB11D8A879B8704
:1033E000AC87BD878091078380930783282F33277D
:1033F00024FD42C023FD7FC020FF11C08881998138
:10340000892B09F486C0888199818F5F9F4F39F09D
:10341000E881F9818481958101969583848322FFD7
:103420007DC020910D838A899B89AC89BD89820FDB
:10343000911DA11DB11D8A8B9B8BAC8BBD8B2091E7
:103440000E838E899F89A88DB98D820F911DA11D34
:10345000B11D8E8B9F8BA88FB98F20910F838A8D82
:103460009B8DAC8DBD8D820F911DA11DB11D8A8FCD
:103470009B8FAC8FBD8F52C08091008382FDFCCFAB
:103480008091008391E6909300832091078391E2DD
:103490009093008310920A8310920B8382FD24C0C4
:1034A00090E082E080930D8382E280930083822FFC
:1034B0008150863408F48FE58093038310920D8346
:1034C000992319F086E28093008380E1809307833B
:1034D0008E859F85A889B9890196A11DB11D8E870A
:1034E0009F87A88BB98B1AC08091078390E08A7060
:1034F000C1F691E0D6CF8AA19BA1ACA1BDA1019656
:10350000A11DB11D8AA39BA3ACA3BDA320FF87CFA0
:1035100075CF8FEF9FEF9983888381CFDF91CF9114
:1035200008950F931F93CF93DF93EC0100E0109168
:103530001F8385E00E94F41310931F8310E004C0E2
:103540001F5F143109F470C082E30E94F41380916C
:10355000078387FFF5CF80910A83803589F78091B3
:103560000B83803769F710920F830FEF0093078367
:1035700081EE8093008380EC8093018310E21093AE
:10358000058310930683109201838FEF0E94F4133A
:1035900081E28093008388E480930E8310920A83F3
:1035A00010920B8310930C8382E080930D8380E450
:1035B000809304838FE58093038386E48093018363
:1035C00080E6809302830093078381E680930083E3
:1035D000A1E0B3E8FE019E012A5F3F4F81918D93E8
:1035E000E217F307D9F7E8E0F3E8119283E8E03156
:1035F000F807D9F786E48093078381E280930083FC
:1036000084E080930C838FEF809307838DE1809318
:103610000F8382E28093008310920D838FEF0E94CC
:10362000F41380E090E006C00F5F043109F07FCF13
:103630008FEF9FEFDF91CF911F910F910895EF9240
:10364000FF920F931F93CF93DF93EC018091590367
:10365000882309F444C00F85188978010894E11C77
:10366000F11CF701A3E6B3E086E00D9001928150D2
:10367000E1F7E989FA8986E211928A95E9F720E073
:1036800033E0AE0163E17CE187E492E00E945913EC
:1036900064EF71E080E090E00E94C410AE0162EE41
:1036A00079E18CE492E00E94101E892BA9F489B77D
:1036B0008F7D89BFF80181819281892B9381892B2C
:1036C00031F489B7806289BF80E090E00DC0C70106
:1036D0000E94911A892BA9F38FEF9FEF05C0CE01AD
:1036E00002960E945631B7CFDF91CF911F910F9173
:1036F000FF90EF900895BF92CF92DF92EF92FF92EA
:103700000F931F93CF93DF938B01FC01C188D28865
:10371000FB01C581D68181859285C80FD91F85851A
:10372000968521893289820F931FC80FD91FF5E032
:10373000CB3EDF0708F06BC0CC33D10508F461C085
:10374000FF2402C00E947E0E8091008382FDFACF8A
:1037500089B78F7D89BFBC2EC0930A838D2F99278F
:10376000E82E80930B831092088380E48093098372
:1037700082E180930083F801658176818381948161
:103780000E94D019F80161857285878190850E9419
:10379000D019F80165857685838594850E94D019B6
:1037A000F80161897289878590890E94D019FF206C
:1037B00051F080E090E02F2D332710921083019676
:1037C00028173907D1F70E94C019B0920583E092FB
:1037D000068380E48093048386E28093008389B724
:1037E000806289BFF60186819781A085B1850196A7
:1037F000A11DB11D86839783A087B18780E090E0EB
:1038000008C02CE3F22EFC1ACCE3D0E09DCF8FEF62
:103810009FEFDF91CF911F910F91FF90EF90DF907D
:10382000CF90BF900895CF93DF93CDB7DEB72497A5
:103830000FB6F894DEBF0FBECDBF1C01FC0147845C
:103840005088A188B28889E00E94F60DF20181813A
:1038500092818923938189238F3F09F4FAC0320131
:103860000894611C711C40E050E060E070E0C5010C
:103870000E94111289B78F7D89BF82E680930083F1
:103880000000000000000000000000000000000038
:103890000000000000000000000000000000000028
:1038A0009091078382E280930083109103831F5FCE
:1038B000103608F016E4191709F484C084E08093E8
:1038C0000A8310920B8310920883109309838AE075
:1038D0008093008300000000000000000000000052
:1038E00000000000000000000000000000000000D8
:1038F00000000000FE0131969E012B5F3F4F80913A
:10390000108381932E173F07D1F70E94C019EB80D7
:10391000FC808F2D992720E0E11021E0820F810F9C
:10392000803608F08A510A818017D1F0982F9F5F66
:10393000903608F09A51901799F089B7806289BF44
:10394000C3010E94911AF501868D978DA0A1B1A1A6
:103950000196A11DB11D868F978FA0A3B1A38ACF19
:10396000C701805490408F5A954018F489818E7019
:1039700069F1CC24DD24802F8150863408F48FE552
:103980008093038389B7806289BFFFEFCF16FFEF73
:10399000DF06B1F2C114D10409F465CFF5018281CB
:1039A0009381A481B5810196A11DB11D828393836A
:1039B000A483B583F201218D328DB601C101F901D5
:1039C000099558CF89B7806289BF4DCF6CEF862E9D
:1039D0006FEF962E8E0C9F1CA40160E180E090E0BA
:1039E0000E945B246C01892B31F280920A83892D1D
:1039F000992780930B8384E0809308831093098335
:103A00008AE08093008300000000000000000000B6
:103A100000000000000000000000000000000000A6
:103A2000000000000000F60183819481892871F074
:103A3000FC01970125503040832F9927982F8091C2
:103A4000108381932150D8F79150C8F70E94C01974
:103A500092CF6DE770E080E090E00E94C410F20128
:103A6000818192818923938189238F3F91F389B743
:103A70008F7D89BF32010894611C711CC3010E94B3
:103A8000911A89B7806289BFEECE9C01FB0189B78C
:103A9000482F55274072507089B78F7D89BF2131DB
:103AA0003105D9F122313105ACF02831310509F465
:103AB00040C029313105BCF12931310509F44DC02F
:103AC0002032310599F585E090E09183808320E0F4
:103AD00030E012C02130310559F02031310579F044
:103AE000232B21F58AB78B7F8ABF8AB7877F8ABF4E
:103AF00080E288BF20E030E0452B89F45BC008B647
:103B000005FE28C081E090E091838083452BF9F089
:103B10008081918180689183808320E030E089B743
:103B2000806289BF47C02231310589F02FEF3FEF16
:103B3000E3CF8AB7982F987083FDC5CF943021F1D9
:103B400081E090E09183808320E030E0D5CF20E0D9
:103B500030E030C011821082D9CF60817181613034
:103B60007105C9F067307105F9F065307105F9F03C
:103B700066307105D9F68AB784608ABF8AB78860D3
:103B80008ABF20E030E0B8CF87E090E09183808367
:103B900020E030E0B1CF8AB78B7F8ABF8AB7877FBA
:103BA0008ABF20E030E0A8CF8AB78460F6CF8AB71A
:103BB0008B7FE3CFC90108951F920F920FB60F922A
:103BC00011242F933F934F935F936F937F938F9322
:103BD0009F93AF93BF93EF93FF938CE492E00E9487
:103BE000021EFF91EF91BF91AF919F918F917F91B5
:103BF0006F915F914F913F912F910F900FBE0F905A
:103C00001F901895CF93DF93DC01EC01EA81FB81D3
:103C1000309719F08D919C910995DF91CF9108957E
:103C2000EF92FF920F931F93CF93DF93EC017B01F1
:103C30008A01EC81FD81309731F060E070E080E036
:103C400090E0099502C080E090E019830883FB8230
:103C5000EA82DF91CF911F910F91FF90EF9008952D
:103C6000CF93DF93EC01EC81FD81309731F060E080
:103C700070E081E190E0099502C08FEF9FEFDF9146
:103C8000CF910895CF93DF93EC01EC81FD813097C4
:103C900031F060E070E082E190E0099502C08FEFC2
:103CA0009FEFDF91CF9108950F931F93CF93DF93F1
:103CB000CDB7DEB724970FB6F894DEBF0FBECDBFE9
:103CC0008C017C836B83FC012481358121153105B6
:103CD000C1F0BE016F5F7F4F80E290E0F90109956E
:103CE000009789F4F80124813581BE016D5F7F4F13
:103CF00081E290E0F9010995009729F489819A8180
:103D000002C08FEF9FEF24960FB6F894DEBF0FBE70
:103D1000CDBFDF91CF911F910F9108950F931F9306
:103D2000CF93DF93CDB7DEB724970FB6F894DEBFFD
:103D30000FBECDBF8C017C836B83FC012481358158
:103D400021153105C1F0BE016F5F7F4F88E190E022
:103D5000F9010995009789F4F80124813581BE01A4
:103D60006D5F7F4F89E190E0F9010995009729F493
:103D700089819A8102C08FEF9FEF24960FB6F89445
:103D8000DEBF0FBECDBFDF91CF911F910F91089580
:103D90000F931F93CF93DF93FC01C189D289EDA9C3
:103DA000FEA909958C01892B49F4CF5BDF4FE8818F
:103DB000F98160E072EC81E090E00995C801DF9143
:103DC000CF911F910F910895CF93DF93EC01EA817A
:103DD000FB810188F289E02D0FB6F8940F9264A55B
:103DE00075A50F900FBE88279927DF91CF91089571
:103DF000CF92DF92EF92FF920F931F93CF93DF93B7
:103E0000EC018B017A0169018C819D8128853985BE
:103E10000FB6F8940F92198618860F900FBE2617CA
:103E2000370769F0232B31F40115110521F580E0E6
:103E300090E028C00097C1F30E945A49F5CF672B44
:103E4000B1F39D838C83998388839B838A83800FBE
:103E5000911F9F838E83FD86EC86DF86CE861B8630
:103E60001A860FB6F8940F92198708870F900FBE25
:103E700080E090E007C0C8010E945D49009709F703
:103E80008FEF9FEFDF91CF911F910F91FF90EF90F8
:103E9000DF90CF900895AF92BF92CF92DF92EF92D2
:103EA000FF920F931F93CF93DF93FB015A01DA0127
:103EB000ED90FD900D911C912E2DEC01C988DA88B2
:103EC000E150F140E732F10540F4EA5BFF4FEE0FBD
:103ED000FF1F0590F491E02D0994CFEFDFEFE7C1CC
:103EE000E1E4F0E0CE0EDF1ED601ED91FC91C801B9
:103EF000B7010995EC01DBC1C3E4D0E0CC0EDD1EB7
:103F0000D601ED91FC910995E501688379838A8357
:103F10009B83C0E0D0E0CBC1E5E4F0E0CE0EDF1E35
:103F2000D601ED91FC91822F0995EC01C0C1C7E447
:103F3000D0E0CC0EDD1ED601ED91FC9109959927BC
:103F4000AA27BB27E50188839983AA83BB83C0E0A6
:103F5000D0E0ADC1E9E4F0E0E1CFCBE4D0E0E9CFDF
:103F6000EDE4F0E0DBCFCFE4D0E0E3CFE6FC8AC1C4
:103F7000C0E0D0E0E7FE0FC0209709F098C1F6013D
:103F80007096268537854485558560857185CF0176
:103F90000E94F81EEC01209709F089C181E590E0AC
:103FA000C80ED91E8FE39FEFAFEFBFEFE822F922D3
:103FB0000A231B2399CFC3E5D0E0CC0EDD1ED6012A
:103FC000ED91FC91CDEADFEFCC0EDD1E09959B0152
:103FD000AC01F5016083718382839383E6018CA534
:103FE0009DA5892B29F42064208331834283538348
:103FF000E6018A8D9B8D892B09F025C1F501808111
:104000009181A281B3818068E50188839983AA8325
:10401000BB83C0E0D0E04BC1F601E086F1860287A9
:104020001387C0E0D0E043C1EE2009F41DC1F601C2
:1040300080819181A281B3818064E6018883998324
:10404000AA83BB83C0E0D0E032C1F60180819181B8
:10405000A281B38186FD4CC0F501108211821282CB
:104060001382C0E0D0E023C1E601EC86FD860E8716
:104070001F87C0E0D0E01BC1E601EDADFEADC80179
:10408000B7010995EC0113C1EFE3F0E0CE0EDF1E9E
:1040900037CFE60188859985AA85BB85FA0180839B
:1040A0009183A283B383C0E0D0E001C1F60184858F
:1040B0009585A685B785EA0188839983AA83BB8302
:1040C000C0E0D0E0F4C0EE2009F4C0C0F601808169
:1040D0009181A281B3818068E60188839983AA8354
:1040E000BB83C0E0D0E0E3C0F601808187FFB4CF9E
:1040F00081E090E0A0E0B0E0E50188839983AA83A5
:10410000BB83C0E0D0E0D3C085E590E0C80ED91EE7
:1041100007CFC7E5D0E00DCFF6017096268537852D
:1041200044855585B701CF010E94F81EEC01892B0B
:1041300009F0BDC0F60183AD94ADFC010995B7C08F
:10414000E601888D998DAA27BB27FA018083918388
:10415000A283B383C0E0D0E0AAC0F601B296268560
:10416000378544855585B701CF010E94F81EEC01C3
:104170009EC0E6018AA59BA5AA27BB27FA018083DA
:104180009183A283B383C0E0D0E091C00FB6F894CE
:104190000F92E601FD8EEC8E0F900FBEC0E0D0E0D6
:1041A00086C0F601848D958DAA27BB27EA018883F6
:1041B0009983AA83BB83C0E0D0E079C00FB6F8949E
:1041C0000F92F601F78EE68E0F900FBEC0E0D0E0A2
:1041D0006EC0E6018E8D9F8DAA27BB27FA018083D2
:1041E0009183A283B383C0E0D0E061C00FB6F8949E
:1041F0000F92E601FFA6EEA60F900FBEC0E0D0E042
:1042000056C0F60186A597A5AA27BB27EA01888391
:104210009983AA83BB83C0E0D0E049C00FB6F8946D
:104220000F92F601F1AAE0AA0F900FBEC0E0D0E015
:104230003EC0E60188A999A9AA27BB27FA01808375
:104240009183A283B383C0E0D0E031C0F6018081C6
:104250009181A281B3818F77E60188839983AA83B4
:10426000BB83C0E0D0E023C0F60180819181A281B0
:10427000B3818F7BE60188839983AA83BB83C0E0E7
:10428000D0E015C0F601B296268537854485558560
:1042900060857185CF010E94F81EEC01892B09F021
:1042A00069CEF60183AD94ADFC01099563CECE01D4
:1042B000DF91CF911F910F91FF90EF90DF90CF9002
:1042C000BF90AF900895CF92DF92EF92FF920F933D
:1042D0001F93CF93DF936C018A01FC01C189D289BE
:1042E00083E0E82EF12CE422F522E114F10491F5AB
:1042F00020EF30E040ED50E060E071E0CE018296CA
:104300000E94F81E892B09F042C086E090E00E94CE
:104310005D499C01892B81F10070107C0050104890
:10432000E9F188819981AA81BB818068888399831A
:10433000AA83BB838901F90111821082D382C282D0
:1043400015821482F1E0EF16F10491F1EBADFCADB2
:1043500009952EC028E330E048E250E060E470E0C8
:10436000CE0140960E94F81E892B71F4F1E0EF1601
:10437000F10409F0BDCFC9CF8C899D890E945A49AB
:104380008EA19FA10E945A490FEF1FEF11C08C8987
:104390009D890E945A490FEF1FEF0AC088819981B9
:1043A000AA81BB818F7788839983AA83BB83C2CF7D
:1043B000C801DF91CF911F910F91FF90EF90DF9097
:1043C000CF900895CF93DF93DC01EC01EA81FB816C
:1043D000C189D28901978E5F9F4F18F08FEF9FEFB1
:1043E00019C0CD010E945A4920E030E040E050E081
:1043F00060E070E0CE0140960E94F81E20E030E0C0
:1044000040E050E060E070E0CE0182960E94F81E2D
:1044100080E090E0DF91CF910895AF92BF92CF926C
:10442000DF92EF92FF920F931F93CF93DF938C0154
:104430005A0120E1E22EF12CE80EF91E0FB6F89495
:104440000F92F70182859385860F971F9387828746
:10445000C285D3850F900FBE4C175D0700F590E124
:10446000C92ED12CCE0CDF1C0BC00FB6F8940F92C6
:10447000F701C285D3850F900FBEAC16BD0678F448
:10448000F80181AD92ADFC010995F801448555858F
:1044900066857785C6010E941112892B31F3CE0102
:1044A000DF91CF911F910F91FF90EF90DF90CF9010
:1044B000BF90AF9008954F925F926F927F928F92CC
:1044C0009F92AF92BF92CF92DF92EF92FF920F93A3
:1044D0001F93CF93DF93CDB7DEB722970FB6F89433
:1044E000DEBF0FBECDBF5A014901FC016188728851
:1044F000B0E14B2E512C460C571CF2018085918562
:10450000892B09F49DC06115710509F4A2C0D3017E
:104510002D913D914D915C910FB6F8940F92F2015F
:10452000C284D3840F900FBE1A141B040CF09AC0DF
:10453000DA01C901F9E0B695A79597958795FA959F
:10454000D1F781708A83E7E056954795379527958F
:10455000EA95D1F7217029838B0160E070E0EE24A9
:10456000FF2421C0F8018491B981B13079F199819A
:10457000923009F446C00F5F1F4F0894E11CF11CF4
:10458000D201ED91FC91119781931196FC93EE93DA
:104590002D913C91F2018681978128173907A1F16D
:1045A000EA14FB04C4F59601260F371FF201868535
:1045B000978528173907A0F46F5F7F4F8114910406
:1045C00089F6D8018C91B981B13089F68A3099F693
:1045D000EA81E13009F438C0F2E0F9838DE0D0CF10
:1045E000F20144855585C3010E940D226C01F20140
:1045F000848595858C159D0508F436C061E070E0D2
:10460000DDCFA1E0A983B7CF848195819183808399
:10461000EA14FB0444F26115710531F10FB6F89408
:104620000F92F20182859385680F791F73876287E5
:104630000F900FBEF30181AD92ADFC01099514C03E
:10464000AFEFEA2EFA2E10C082E08A8389838DE0D4
:1046500097CF40E050E060E070E0C3010E940D227F
:104660007C0102C0EE24FF24C70122960FB6F89405
:10467000DEBF0FBECDBFDF91CF911F910F91FF9095
:10468000EF90DF90CF90BF90AF909F908F907F90F2
:104690006F905F904F90089521E030E0FC0182819F
:1046A00093810E945B22089520E030E0FC0182812A
:1046B00093810E945B220895AF92BF92CF92DF92C6
:1046C000EF92FF920F931F93CF93DF937B015A01D9
:1046D000EC01EA81FB8101891289E801A2966885D3
:1046E00079856115710509F1E114F10409F492C0AD
:1046F0000FB6F8940F924A855B850F900FBE411557
:104700005105B1F4F80183AD94ADFC010995F801B0
:104710004085518562857385CE0140960E941112B5
:10472000892B31F380E090E090C08FEF9FEF8DC038
:10473000D701F801808187FF4DC0CC24DD24EE2411
:10474000FF247AE00BC06A30F1F0F80114AA6D93EF
:104750000894C11CD11C0894E11CF11CCA14DB0490
:1047600008F066C0E416F50609F1EA81FB81619163
:10477000FB83EA832A813B818E819F812817390739
:1047800079F06D3001F7F80184A9882311F06817DA
:1047900011F7F80164AB7D930894C11CD11CDBCFE9
:1047A0008C819D819B838A83ECCF76010FB6F89430
:1047B0000F928A859B858E199F099B878A870F9008
:1047C0000FBE2A853B858C859D8528173907C0F14A
:1047D000C6013BC06A01A416B50680F1C114D1041C
:1047E000B9F3AD014C0D5D1D03C0A417B507E9F287
:1047F000EA81FB8181918D93FB83EA832A813B814E
:104800008E819F812817390781F78C819D819B8339
:104810008A83EBCF2E853F854C855D85CE010E9436
:10482000F81EE801EBADFCAD099580E090E00DC00D
:10483000E114F10409F0BACFC60107C06501CECF7B
:10484000E801EBADFCAD0995C601DF91CF911F9159
:104850000F91FF90EF90DF90CF90BF90AF900895B1
:104860000F931F938C01FC01808191810E94610C48
:10487000F80111821082138212821F910F91089504
:104880000F931F93CF93DF93EC018B01CB010E9419
:10489000E30B99838883892B29F01B830A8380E0AB
:1048A00090E004C01B821A828FEF9FEFDF91CF91BF
:1048B0001F910F910895BF92CF92DF92EF92FF92D6
:1048C0000F931F93CF93DF937C01B62EEA01892BC0
:1048D00009F469C0BB2009F4D5C0209799F4F70109
:1048E00002810B21C02FDD27C4FD58C0C5FD51C07A
:1048F000C6FD4AC007FDB3C00095F7018281802341
:104900008283C0C0CB2CDD24C4FE1AC0F7012281F3
:1049100024FF69C0858196818C179D0720F0F701DF
:10492000D683C5830FC087010D5F1F4FC8010E944A
:104930003024BE01C8010E944024892B09F05BC0CD
:10494000F7012281C5FE0CC025FF5BC0F701818500
:1049500092858C179D0708F468C0F701D287C1873C
:10496000C6FE0CC026FF57C0F701858596858C17BB
:104970009D0708F467C0F701D687C587B7FC1CC040
:104980002B29F70122837EC0C7010B960E94302499
:10499000B1CFC70107960E943024AACFC701039662
:1049A0000E943024A3CF83E190E00E94E30C7C01BD
:1049B000892B09F08FCF66C027FD0AC0BE01C70151
:1049C0000F960E944024892BB1F4F7012281D8CFA1
:1049D000F701818992898C179D0708F445C0F7017A
:1049E000D28BC18BCDCFBE01C70103960E9440245C
:1049F000892B09F4A5CFC7010E944D25EE24FF2481
:104A000041C0BE01C70107960E944024892B99F737
:104A1000F7012281A5CFBE01C7010B960E94402459
:104A2000892B49F7F7012281A9CF8701095F1F4F21
:104A3000C8010E943024BE01C8010E944024892B75
:104A400039F3D9CF8701055F1F4FC8010E94302479
:104A5000BE01C8010E944024892B21F3CCCFC7019D
:104A60000F960E94302448CF8701015F1F4FC80175
:104A70000E943024BE01C8010E944024892B09F401
:104A8000A4CFB9CFC701DF91CF911F910F91FF90B4
:104A9000EF90DF90CF90BF900895CF93DF93EC011C
:104AA000009751F040E050E06A810E945B24CE0103
:104AB0000E94610C892B19F480E090E002C08FEF16
:104AC0009FEFDF91CF910895EF92FF920F931F9385
:104AD000CF93DF938C0183E190E00E94E30CEC0123
:104AE000009709F476C07C01F80165817681611533
:104AF000710541F5F8016185728561157105D1F582
:104B0000F801658576856115710509F04CC0F801DD
:104B1000618972896115710509F462C0CE010F9631
:104B20000E944024892B09F051C0F80167857089E3
:104B3000418952898F8598890E94164A8A818068A6
:104B40008A834EC003960E944024892B09F044C0FA
:104B5000F80163817481458156818B819C810E941B
:104B6000164A8A8180618A83F801618572856115A0
:104B7000710531F2CE0107960E944024892B31F550
:104B8000F80167817085418552858F8198850E94E3
:104B9000164A8A8180628A83F80165857685611567
:104BA000710509F4B4CFCE010B960E944024892BE5
:104BB00069F4F80163857485458556858B859C85E8
:104BC0000E94164A8A8180648A83A1CFCE010E9406
:104BD0004D25EE24FF2404C0CE010E944D25F9CFBF
:104BE000C701DF91CF911F910F91FF90EF90089532
:104BF0000E94FE2508950E941D260895CF93DF93FD
:104C000041155105A9F09C01E0E0F0E0EB01D9016C
:104C10000E94914A802D9991981721F0D901092E6F
:104C20000E94994A31962F5F3F4F4E175F0779F7E1
:104C300080E090E0DF91CF910895CF93DF93EA0178
:104C4000DC01FB01219724F00E94914A0192FACFE6
:104C500080E090E0DF91CF9108950F931F93CF9361
:104C6000DF938C01C091BC02D091BD02209789F1E5
:104C7000FE0105C00190F081E02D309711F1808D8B
:104C8000918D08171907B1F7828D938DA48DB58D7D
:104C900082179307A407B50769F7868D978D861746
:104CA000970741F78389882329F3CF0116C0888DA0
:104CB000998D8017910781F00990D881C02D209798
:104CC00041F08B89813099F30990D881C02D2097CC
:104CD000C1F780E090E001C0CE01DF91CF911F913C
:104CE0000F910895CF93DF93FC01EA01892BB1F076
:104CF00080E16230780759F180E1633078078CF009
:104D000080E16530780709F442C06650704169F16E
:104D1000E05AFF4F8AE397E2918380838FEF9FEF02
:104D20005DC06230710509F444C06150704181F783
:104D3000452B21F02230310509F44AC0E05AFF4FDB
:104D400086E190E0918380838FEF9FEF47C0452BF2
:104D5000A9F32230310591F7E85BFF4F8081918103
:104D60009983888380E090E039C0452B39F3243063
:104D7000310521F7EA59FF4F80819181A281B381EA
:104D800088839983AA83BB8380E090E027C0452B6A
:104D9000A9F22430310591F6E659FF4F80819181C7
:104DA000A281B38188839983AA83BB8380E090E04A
:104DB00015C0452B19F22230310509F0BFCFEE5A4C
:104DC000FF4F808191819983888380E090E006C0C5
:104DD000818992899983888380E090E0DF91CF91E7
:104DE0000895FC01892B29F0E05AFF4F80819181C1
:104DF000089586E397E20895CF93DF93DC01EA01FB
:104E00006A30710561F06A3071051CF48FEF9FEF15
:104E100025C06B307105B9F06C307105B9F7FD0133
:104E2000E65BFF4FAA5BBF4F8D919C912081318142
:104E3000821B930BAA27BB2788839983AA83BB83F2
:104E400080E090E00BC0FC0185859685AA27BB27F2
:104E500088839983AA83BB8380E090E0DF91CF9120
:104E600008950F931F93CF93DF938C01EC01C45BE4
:104E7000DF4FE881F981309759F0808191819983E2
:104E80008883CF010E944D25E881F9813097A9F7E9
:104E9000E801E8ADF9AD309761F080819181E801DA
:104EA00099AF88AFCF010E944D25E8ADF9AD30979D
:104EB000A1F7E801C05BDF4FE881F981309759F035
:104EC0008081918199838883CF010E944D25E8815B
:104ED000F9813097A9F7DF91CF911F910F91089534
:104EE0002F923F924F925F926F927F928F929F92FA
:104EF000AF92BF92CF92DF92EF92FF920F931F93E8
:104F0000CF93DF93CDB7DEB726970FB6F894DEBF09
:104F10000FBECDBF6C011B012A010E947E0EC11481
:104F2000D10409F447C0F6018389843021F08389D4
:104F3000853009F0B4C02114310481F141145104C9
:104F400069F196E4692E712C6C0C7D1CF601E65B10
:104F5000FF4FFA83E98386E6E82EF12CEC0CFD1C6A
:104F60008601025B1F4FF30180819181A981BA8183
:104F70000D90BC91A02DBE83AD838A179B07E9F4E9
:104F8000F6018389843069F4D7014D915D916D916B
:104F90007C91C8010E941112892B29F340E050E056
:104FA000BDC0E0E6F0E0CE0EDF1E89E497E2D60158
:104FB0008D939C934FEF5FEFB1C08A1B9B0B8415C1
:104FC000950520F4009709F474C02C01AA24BB2491
:104FD000C601845B9F4F9C838B832EC0678570893D
:104FE000620F731FA701C1018A0D9B1D0E94164A03
:104FF000AE0CBF1C6D817E816E0D7F1D7E836D8327
:10500000E016F106B0F0D4018D919C91EB81FC810A
:1050100091838083D3018D919C911197ED81FE81C5
:105020008E1B9F0B8D939C93C4010E944D251E8265
:105030001D82A414B50438F5EB81FC818080918039
:10504000F401018912892D813E81021B130B72012B
:10505000EA18FB080E151F0508F6F401678570892C
:105060002D813E81620F731FA801C501820D931D22
:105070000E94164AA00EB11E6D817E81600F711FC5
:105080007E836D83C0CFED81FE81A981BA81ED93CE
:10509000FC93F6018389843081F0A2013FC020E6B1
:1050A00030E0C20ED31E89E497E2D6018D939C9323
:1050B00081CF44245524A20131C0EC5BFF4F4081D5
:1050C000518128E430E0C20ED31ED6012D913C91CF
:1050D00068EB7FEFC60ED71ECA01840D951D2817F9
:1050E000390708F4C901A2E5B0E0CA0EDB1ED601FB
:1050F0002D913C916EEA7FEFC60ED71E241735071F
:1051000018F02817390720F091838083A20106C088
:1051100091838083C6010E949534A201CA0126961C
:105120000FB6F894DEBF0FBECDBFDF91CF911F91B8
:105130000F91FF90EF90DF90CF90BF90AF909F9036
:105140008F907F906F905F904F903F902F90089539
:105150000E9470270895CF92DF92EF92FF920F93F3
:105160001F93CF93DF93EC016B018A010E947E0EA7
:10517000209709F447C0C114D104B9F101151105F4
:10518000A1F172E5E72EF12CEC0EFD1EF7018081F6
:1051900091818017910760F18B89843069F549A569
:1051A0005AA58DA19EA1481B590B9A0136952795AA
:1051B00036952795F701808191812817390738F4B2
:1051C0008DA99EA9841B950B80179107F0F4C659F1
:1051D000DF4F488159816A817B81CA56D040CE0118
:1051E000CA960E941112892BB9F240E050E018C013
:1051F0008C018B89843099F2C05ADF4F89E497E2A1
:10520000998388834FEF5FEF0BC088A1806188A3EB
:10521000A801B601CE010E942232892B99F7A8017C
:10522000CA01DF91CF911F910F91FF90EF90DF9016
:10523000CF900895CF92DF92EF92FF920F931F933A
:10524000CF93DF936C017B018A0114161506BCF421
:10525000C0E0D0E005C0C80FD91FC017D1078CF43B
:10526000A8014C1B5D0BB7016C0F7D1FC6010E948E
:10527000AB28181619067CF3CFEFDFEF02C0C0E0B1
:10528000D0E0CE01DF91CF911F910F91FF90EF9071
:10529000DF90CF900895AF92BF92CF92DF92EF92BE
:1052A000FF920F931F93CF93DF93EC017B018A0151
:1052B000892B09F492C08B89843009F091C0411583
:1052C0005105E1F05B012D853E8521153105E9F49D
:1052D00069897A894617570708F05BC06A01CB01D4
:1052E0000E94E30B988B8F87009709F476C0A60184
:1052F000B5010E94164ADE86CD8699C04D855E8531
:105300004115510509F493C05AC049895A89C90108
:10531000800F911F8417950770F16A01C21AD30A92
:105320008F859889A601820F931F0E94164A49898A
:105330005A896F857889CE010E941A2999230CF425
:105340006EC05701AC0CBD1C98012C193D09698930
:105350007A892617370708F051C07901E114F10462
:1053600009F447C0A701B5018F8598890E94164AA4
:10537000FE86ED865CC08F859889A801820F931FF9
:105380000E94164A8D859E85800F911F9E878D876E
:105390004EC0CA010E945B4A6C015801A81AB90AA2
:1053A000A501B701CE010E941A2997FD16C0C114AC
:1053B000D104E9F1AE0CBF1C69897A8990CF6F8561
:1053C0007889CE010E941A2999234CF18F859889FA
:1053D0000E94610C1E861D862AC00FEF1FEF27C09A
:1053E000C05ADF4F89E497E2998388830FEF1FEF5C
:1053F0001EC08F8598890E94610CBACFC8010E9497
:105400005B4A7C016901C81AD90AA601B501CE011F
:105410000E941A2997FD03C0AC0CBD1C9FCF8F853D
:1054200098890E94610C1E861D860FEF1FEFC80130
:10543000DF91CF911F910F91FF90EF90DF90CF9070
:10544000BF90AF900895CF92DF92EF92FF920F93AB
:105450001F93CF93DF936C017B01EA014115510546
:10546000A1F0CA010E94E30B8C01009771F0AE011C
:10547000B7010E940D4AAE01B801C6010E944B2936
:10548000EC01C8010E94610C07C0AE0160E070E051
:10549000C6010E944B29EC01CE01DF91CF911F91F3
:1054A0000F91FF90EF90DF90CF9008950F931F938F
:1054B0008C0140E050E060E070E00E944B29C801A0
:1054C0000E94E83C1F910F9108950F931F93CF9373
:1054D000DF93EC018A01892BB1F080E1623078071B
:1054E00059F1E0E163307E078CF080E165307807A8
:1054F00009F449C06650704191F1C05ADF4F8AE308
:1055000097E2998388838FEF9FEF7DC062307105AA
:1055100009F44DC06150704181F7452B21F02230D4
:10552000310509F459C0C05ADF4F86E190E09983F4
:1055300088838FEF9FEF67C041155105A1F322309B
:10554000310589F7FA0180819181C85BDF4F99832A
:10555000888324979983888380E090E054C0411524
:10556000510509F324303105F1F6CA59DF4FFA012C
:1055700080819181A281B38188839983AA83BB832F
:1055800080E090E040C04115510569F224303105BA
:1055900051F6C659DF4FFA0180819181A281B38112
:1055A00088839983AA83BB8380E090E02CC0411557
:1055B000510509F4B8CF2230310509F0B4CF8B89F9
:1055C0008823C9F4CE5ADF4FFA01808191819983F3
:1055D000888380E090E017C040E050E060E070E039
:1055E000CE010E944B29F801808191819A8B898B91
:1055F00080E090E008C0C05ADF4F88E497E29983CA
:1056000088838FEF9FEFDF91CF911F910F910895C6
:10561000CF93DF938091BE02882359F40E94133404
:1056200020E0892B09F450C02093BE02222309F404
:1056300051C082E790E00E94E30C009709F44AC051
:10564000EC011B8A84E08C8388EA98E29E838D8338
:105650008BE499E298878F8383E29AE29A8789871D
:105660008CEF96E29C878B870E94FF0E69A37AA33A
:105670008BA39CA36DA37EA38FA398A769A77AA7EA
:105680008BA79CA7CC5BDF4F80E99CE09983888344
:105690002496998388832A9628E132E039832883E7
:1056A000269688EE93E099838883C855D0408091F0
:1056B000BC029091BD02998388833A8B298BD09349
:1056C000BD02C093BC0208C021E02093BE02222389
:1056D00009F0AFCFC0E0D0E0CE01DF91CF910895C7
:1056E000CF93DF93EC01E091BC02F091BD023097C3
:1056F00079F1E817F90729F424C0C817D90731F060
:10570000FC01808191810097C1F722C08881998135
:1057100091838083CE010E9431278D859E85892BC0
:1057200049F482E7FE0111928A95E9F7CE010E94C1
:10573000610C0EC08F8598890E94610C1E861D86A3
:10574000F0CF888199819093BD028093BC02E2CF13
:10575000DF91CF910895FC01062E672F702D718F78
:10576000608F0E94F2350895CF92DF92EF92FF9200
:105770000F931F93CF93DF936C017A018B01A901E3
:10578000009709F47AC0EC018B89813009F484C058
:10579000F6018389882309F073C0E091BC02F0917F
:1057A000BD0260E070E18091520290915302019637
:1057B000909353028093520280915202909153022F
:1057C000892B21F47093530260935202309701F1B8
:1057D0008091520290915302082E892F902D208D96
:1057E000318D82179307F9F2DF010D90BC91A02D46
:1057F000109771F08091520290915302082E892FD8
:10580000902DED01288D398D2817390761F2EDCFE4
:105810008091520290915302082E892F902DF6010B
:10582000918F808F042E452F502DE6015F8F4E8F74
:10583000E28EF38E048F158F40E050E0C801B7016F
:105840000E94B72CFC01892B79F00784F089E02DA8
:1058500087819085A185B2858C8B9D8BAE8BBF8B0C
:10586000C6010E94D43523C0E0E6F0E0CE0EDF1E74
:1058700081E597E2E601998388838FEF9FEF17C058
:1058800080E690E0C80ED91E88E497E2E60199838D
:1058900088838FEF9FEF0BC0E0E6F0E0CE0EDF1EB7
:1058A0008DE397E2E601998388838FEF9FEFDF9185
:1058B000CF911F910F91FF90EF90DF90CF900895BF
:1058C000CF92DF92EF92FF920F931F93CF93DF93CC
:1058D0007B018C016A01622F2430A8F5C091570327
:1058E000D0915803FE01209731F437C00190F08128
:1058F000E02D309791F186819781A085B1858E2129
:105900009F21A023B12322813381448155818217B5
:105910009307A407B50751F7C114D10449F02285B4
:10592000338544855585211531054105510571F4AF
:1059300086859785892B89F46F5FE284F3840485DB
:105940001585643079F6E0E0F0E007C0D6012D93CC
:105950003D934D935C931397EBCFCF01DF91CF91A4
:105960001F910F91FF90EF90DF90CF900895FA0173
:10597000452B21F010821182128213826F3F2FEF8C
:1059800072072FEF82072FEF920751F020E0AF014F
:105990000E94602CFC01309749F086859785089518
:1059A000E0915703F09158033097B9F780E090E009
:1059B00008954F925F926F927F928F929F92AF92D3
:1059C000BF92CF92DF92EF92FF920F931F93CF93EC
:1059D000DF93CDB7DEB724970FB6F894DEBF0FBEC6
:1059E000CDBF2B013C0149015A01E982FA820B83A8
:1059F0001C83E0905703F0905803E114F10409F47C
:105A000045C0F70186819781A085B18528173907A0
:105A10004A075B0758F03AC0F70186819781A08555
:105A2000B18588169906AA06BB0638F48701D70106
:105A3000ED90FC90E114F10479F780E190E00E9490
:105A4000E30B9C010097F9F0482059206A207B2045
:105A5000FC01428253826482758286829782A0868C
:105A6000B18689819A81AB81BC8182879387A48723
:105A7000B587D786C686F182E082D8012D933C9304
:105A800080E090E006C08FEF9FEF03C007E513E0D2
:105A9000D4CF24960FB6F894DEBF0FBECDBFDF91F2
:105AA000CF911F910F91FF90EF90DF90CF90BF901B
:105AB000AF909F908F907F906F905F904F900895E0
:105AC000CF93DF93EC0119821882E0915703F09194
:105AD0005803309751F080E090E00190F081E02D84
:105AE00001963097D1F7998388838881998182952F
:105AF0009295907F9827807F98270E94E30B0097CC
:105B0000A1F0C0915703D0915803209781F0DC0198
:105B1000FE0120E101900D922150E1F7409609909D
:105B2000D881C02D209799F702C019821882DF9181
:105B3000CF9108954F925F926F927F928F929F9232
:105B4000AF92BF92CF92DF92EF92FF920F931F938B
:105B5000CF93DF934B015C0129013A01E091570398
:105B6000F0915803EF013097E1F12FEF3FEF09C0BB
:105B7000E881F981EF01F0935803E09357033097E0
:105B800091F182819381A481B58188159905AA0537
:105B9000BB0571F786819781A085B1858415950530
:105BA000A605B70529F782859385A485B5858E1549
:105BB0009F05A007B107E1F6868597858C159D05A1
:105BC000B9F6C081D181D0935803C0935703CF0158
:105BD0000E94610C20E030E0C0915703D09158033F
:105BE000C7CF2FEF3FEFC901DF91CF911F910F91E9
:105BF000FF90EF90DF90CF90BF90AF909F908F90ED
:105C00007F906F905F904F900895CF93DF93EC015A
:105C1000E0915703F09158033097F1F0868597850E
:105C20008C179D0779F0209769F08081918190937E
:105C3000580380935703E0915703F091580330972E
:105C400069F70AC08081918190935803809357032C
:105C5000CF010E94610CDCCF80E090E0DF91CF911A
:105C60000895CF93DF93CDB7DEB724970FB6F8949E
:105C7000DEBF0FBECDBFFC0119821A821B821C82BF
:105C8000DE01119650E04081842F80538A30F8F471
:105C900020E030E0C901880F991F880F991F880FF5
:105CA000991F220F331F280F391F842F992787FD33
:105CB0009095280F391F2053304031964081403352
:105CC0005CF04A334CF42F3F310521F318F36FEFAA
:105CD0007FEF8FEF9FEF14C02F3F310509F0B8F72A
:105CE0005F5F2C9380818E3229F4543081F31196BA
:105CF0003196C9CF543059F769817A818B819C8163
:105D000024960FB6F894DEBF0FBECDBFDF91CF91C2
:105D10000895AF92BF92CF92DF92EF92FF920F93CE
:105D20001F93CF93DF93CDB7DEB727970FB6F894C5
:105D3000DEBF0FBECDBF6C837D838E839F83F4E077
:105D4000CF2ED12CCC0EDD1EA0E00FEB12E0BB2439
:105D50007E010894E11CF11CEEE2AE2EF6012081DA
:105D6000822F6AE00E944F4A382F80834A2F55279E
:105D7000F701E40FF51F822F0E944F4A905D908338
:105D80008A2F8F5F3323D1F49A2FAF3F61F0D80170
:105D9000F701E90FF11D80818D939150C8F7040F31
:105DA000151F0F5F1F4FF801A1928F01B394F3E00D
:105DB000FB1530F00894C11CD11C80E0A82FCECF79
:105DC00001501040F80110828FEB92E027960FB639
:105DD000F894DEBF0FBECDBFDF91CF911F910F9121
:105DE000FF90EF90DF90CF90BF90AF900895CF934A
:105DF000DF939C01EB01EB81FC813E96F887EF83FA
:105E00003E978D819E810E979A8789878EE090E0DC
:105E10009E838D8384859585082E892F902D48E05B
:105E20008030940739F08650984041F0CB010E94B1
:105E30004D2507C0C9010E94F73D03C0C9010E945A
:105E40008B43DF91CF9108958F929F92AF92BF9233
:105E5000CF92DF92EF92FF920F931F93CF93DF9336
:105E60004C018B016A0179014EE050E060E1C9010B
:105E70000E945B24892B61F1F701C381D481F40175
:105E8000A784B088DE011696F501319686E0019070
:105E90000D928150E1F7C114D104E9F0DE01F60161
:105EA00086E001900D928150E1F7002E012F102D18
:105EB0001D870C87E501EB8DFC8DB701C4010995A9
:105EC000892B19F480E090E00EC0C7010E944D2597
:105ED0008FEF9FEF08C046E050E06FEF70E0CE011B
:105EE0000E941F4AE2CFDF91CF911F910F91FF9047
:105EF000EF90DF90CF90BF90AF909F908F900895DC
:105F00002F923F924F925F926F927F928F929F92C9
:105F1000AF92BF92CF92DF92EF92FF920F931F93B7
:105F2000CF93DF93CDB7DEB72A970FB6F894DEBFD5
:105F30000FBECDBF1C012A013B0148015901CD8292
:105F4000DE82EF82F886FC010784F089E02DFA8773
:105F5000E987411551056105710509F4B0C0E9856E
:105F6000FA85478250866186728681149104A10465
:105F7000B10409F49DC0E985FA858786908AA18AD3
:105F8000B28AA3019201282139214A215B21298368
:105F90003A834B835C836101EE24FF248701A501D2
:105FA000940169817A818B819C810E94D92C8D8199
:105FB0009E81AF81B8850097A105B10509F06BC03E
:105FC000AAE5B3E0F101329689E001900D9281508B
:105FD000E1F7E985FA858181882321F4828188238C
:105FE00009F448C0A3E6B3E0E985FA85319686E076
:105FF00001900D928150E1F74092690350926A033B
:1060000060926B0370926C0380926D0390926E03AA
:10601000A0926F03B09270032D813E814F8158850D
:10602000211531054105510579F08D819E81AF81A2
:10603000B8858093710390937203A0937303B09318
:1060400074030E9443314BC080917103909172039D
:10605000A0917303B091740388219921AA21BB21D7
:1060600029813A814B815C81281739074A075B07F0
:10607000E1F6E7CF8381882309F0B4CF84818823B8
:1060800009F0B0CF8581882309F0ACCF86818823C1
:1060900009F4B2CFA7CF7C018D0120E030E040E0D1
:1060A00050E060E070E080E090E00E94D92C88CF62
:1060B00084E592E00E94312E4B015C015CCF409060
:1060C000690350906A0360906B0370906C034114F5
:1060D00051046104710409F042CF8FEF9FEF2A96BB
:1060E0000FB6F894DEBF0FBECDBFDF91CF911F91E9
:1060F0000F91FF90EF90DF90CF90BF90AF909F9067
:106100008F907F906F905F904F903F902F90089569
:106110002F923F924F925F926F927F928F929F92B7
:10612000AF92BF92CF92DF92EF92FF920F931F93A5
:10613000CF93DF93CDB7DEB724970FB6F894DEBFC9
:106140000FBECDBF7C836B8319012A013701480143
:106150000E949112FC01009719F48FEF9FEF64C029
:106160009A83898383858330C1F7A785B0898C9111
:10617000863091F41196EB81FC8101900D92815053
:10618000E1F77601650194018301B201A1018981E2
:106190009A810E94802F48C08731F9F6A188B28881
:1061A000F50121A232A243A254A2E114F104010597
:1061B000110541F48FEF682E8FEF782E8FEF882E28
:1061C0008FEF982EF50161A672A683A694A6C5014D
:1061D0000E94A911F501FF96AE014F5F5F4F67E185
:1061E00071E0808191810E94334740E65AEE60E081
:1061F00070E0C5010E941112892B09F0AECFF501A4
:1062000084AD893009F0A9CFC5A0D6A0E7A0F0A43D
:1062100001A512A523A534A541A152A163A174A192
:1062200089819A810E94802F24960FB6F894DEBF50
:106230000FBECDBFDF91CF911F910F91FF90EF90D7
:10624000DF90CF90BF90AF909F908F907F906F9096
:106250005F904F903F902F900895AF92BF92CF9252
:10626000DF92EF92FF920F931F93AA24BB24650144
:106270000E9488301F910F91FF90EF90DF90CF9098
:10628000BF90AF90089580E28093590340E250E0C0
:1062900069E573E080E490E00E94F825892B19F409
:1062A00080E090E008958FEF9FEF08950F931F9384
:1062B000CF93DF938C01C9E5D3E040E250E0BE010B
:1062C00080E490E00E94FB25892BB9F4809159036A
:1062D000803239F4B801CE0101960E94264A892BFA
:1062E00079F080E219928A95E9F746E050E06FEF85
:1062F00070E083E693E00E941F4A8FEF9FEF02C099
:1063000080E090E0DF91CF911F910F910895AF92BF
:10631000BF92CF92DF92EF92FF920F93CF93DF93D2
:106320006C01FC01A780B084C385D4858D8582FD76
:1063300050C0F601128A118A84E190E09687858721
:10634000288139818A819B81998388833B832A8331
:106350008D85992784FF41C084E08D878885998544
:10636000AA85BB858C839D83AE83BF8318861986DF
:106370001A861B8680E58C871F861E861B8A1A8AD2
:10638000198A188AF601E584F6840E2CEF2CF02C7D
:10639000F50124853585468557856089718982890F
:1063A000938906E00E94C03DDC01CB01F6014585E2
:1063B0005685BE010E94BB3D998B888BF5014485B3
:1063C000558566857785960186E00E94113F892B69
:1063D00069F5C6010E944D2529C081FF1EC08C8130
:1063E0009D81AE81BF81082E8B2FB02D092E9A2F53
:1063F000A02D0196A11DB11D082E8B2FB02D092EA9
:106400009A2FA02D88879987AA87BB871C821D8217
:106410001E821F8284E18D87ADCF8C819D81AE81EC
:10642000BF8188879987AA87BB87F0CF80E090E0FB
:10643000DF91CF910F91FF90EF90DF90CF90BF90C1
:10644000AF9008956F927F928F929F92AF92BF927A
:10645000CF92DF92EF92FF920F93CF93DF93CDB75E
:10646000DEB722970FB6F894DEBF0FBECDBF6C012A
:106470007B013A01452B09F0DCC0FC0190A1892F7A
:106480008B7009F4D3C091FFD8C008E148E150E017
:1064900060E480E090E00E945B244C01009709F4E6
:1064A00074C1FC01A384B484F601808D918DF50143
:1064B00091838083F601868D978DF5019383828386
:1064C000000F000F0487F60180A1877F80A381A5BC
:1064D00092A5A3A5B4A5082E8B2FB02D092E9A2F17
:1064E000A02DF50184839583A683B783F60180A14F
:1064F00084FFD9C080E1F5018587F60180A18F7EF8
:1065000080A320E430E0C20ED31EF6018081918189
:10651000A281B38120EC3FEFC20ED31E082E8B2F39
:10652000B02D092E9A2FA02DF50180879187A28783
:10653000B387F60180A1992781FDFFC06114710422
:1065400009F0C3C080FFBDC0F501858581608587E6
:10655000F60180A18E7F80A381A592A5A3A5B4A5F5
:106560000196A11DB11D81A792A7A3A7B4A7A6015B
:106570004E5A5F4F24E430E0C20ED31EF601208154
:1065800031818CEB9FEFC80ED91EFA018081918179
:106590002817390708F08EC0F50117861686F50111
:1065A000118A108A138A128AF401E584F68481899B
:1065B0009289E80EF91E0E2CEF2CF02CF601228D9C
:1065C000338D448D558D648975898689978906E058
:1065D0000E94C03DDC01CB01F40145855685B50123
:1065E0000E94813DF40141895289678570890E942A
:1065F000BB3DF501918B808B672819F5858599271F
:1066000083709070892BE9F47401F601428D538DEB
:10661000648D758D970186E00E94113F892B19F0DA
:106620008FEF9FEFBDC0C7010E944D2580E090E035
:10663000B7C0FC0190A191FD28CF04E144E150E0F6
:1066400027CFF40111821082F601A0ADB1AD1097F1
:1066500011F463C0DC018D919C9111970097D1F7E3
:106660008D929C9296012C5A3F4FF9018081918125
:10667000A281B3810097A105B10581F4F501848160
:106680009581A681B781082E8B2FB02D092E9A2FC8
:10669000A02DF90180839183A283B383C4010E945A
:1066A00064257C01B2CFF50115861086118612860D
:1066B00013863FCF022E232F302DF50137872687F3
:1066C0006ECFA6014E5A5F4F55CFA30160E8C401BB
:1066D0000E945B244C01009709F457C0A301B70145
:1066E000FC01878590890E94164AC301AA27BB270F
:1066F000F60121A532A543A554A5280F391F4A1F2D
:106700005B1F21A732A743A754A7F50185858860A1
:106710008587A6014E5A5F4F2DCF91AE80AE0E9465
:106720000D0F2EE530E0C20ED31EF601718360839B
:1067300022EA3FEFC20ED31E95CFA6014E5A5F4FFD
:10674000FA0180819181082E892F902D9A83898367
:10675000F501858582608587F60180A18D7F80A304
:1067600081A592A5A3A5B4A50196A11DB11D81A7E0
:1067700092A7A3A7B4A782E0F501848B84E0858B60
:106780008981868B8A81878BF5CE20E630E0C20E28
:10679000D31E87E497E2F601918380838FEF9FEF0A
:1067A00022960FB6F894DEBF0FBECDBFDF91CF911A
:1067B0000F91FF90EF90DF90CF90BF90AF909F90A0
:1067C0008F907F906F900895CF93DF93EC01C05A24
:1067D000DF4F798368831A921A921A921A92CC55D3
:1067E000D0408B89863018F08AE08B8B01C01B8AE1
:1067F000CE010E943127CE01825B9F4F0E94A911DA
:10680000CE01CA960E94A911CE018E599F4F0E94B7
:10681000A911CE018C599F4F0E94A91180E090E0F0
:10682000DF91CF9108958091CF029091D002892B72
:1068300019F080E090E0089520E032E040E050E080
:1068400065ED77E382E692E00E9459139093D002BF
:106850008093CF02892B69F78FEF9FEF0895CF9236
:10686000DF92EF92FF920F931F93CF93DF936C0110
:10687000FC01118210828091CF029091D002892B6D
:1068800009F447C0E0907903F0907A03E114F10431
:10689000B9F1F601C185D28585859685C80FD91FC6
:1068A00081899289C80FD91FC050D84F0091D10259
:1068B0001091D2020C0F1D1FC050D8400E94DE0C58
:1068C00008171907C8F48091D1029091D2028C0F59
:1068D0009D1F9093D2028093D10201C07C01F701E9
:1068E000808191810097D1F7F701D182C0828BE737
:1068F00093E00E94B41110C0C6010E944D250CC047
:10690000D0927A03C09279038BE793E00E94B4118E
:1069100003C0C6010E948731DF91CF911F910F9173
:10692000FF90EF90DF90CF900895FC01892B69F0E4
:1069300080A1886180A340E050E060E070E0CF017A
:106940000E94223280E090E008958FEF9FEF08953B
:10695000EF92FF920F931F93CF93DF93EC018B0184
:10696000DC01A45BBF4FED91FC911197309711F4BE
:1069700046C0FC01808191810097D9F71183008383
:10698000DE01AA5BBF4F8D919C911197F80121897F
:106990003289820F931F8D939C9380E4E82EF12C13
:1069A000EC0EFD1E618972899B0144275527F70172
:1069B00080819181A281B381820F931FA41FB51F93
:1069C00080839183A283B383FE01EC5BFF4F8081C0
:1069D00091816817790770F01182108228A1822FA7
:1069E000806188A3F80180819181892B59F01182FF
:1069F00010820AC0861B970B91838083EFCF6D9323
:106A00007C93BECF286128A340E050E060E070E0B6
:106A1000CE010E942232DF91CF911F910F91FF9002
:106A2000EF9008951F93CF93DF93EC01162F8B897E
:106A3000853009F443C0863030F1883009F189305F
:106A400008F43FC0893009F493C08A30C9F080E06F
:106A50001B8B882371F140E050E060E070E0CE01D4
:106A60000E942232892B29F1123019F5C05ADF4FCA
:106A700080E597E299838883CE0104960E942211D3
:106A80002FEF3FEF8CC0823009F440C0833010F10B
:106A9000833009F454C08430D1F6653009F44AC01B
:106AA000663071F788A1816188A381E01B8B882300
:106AB00091F61530D9F020E030E071C0683001F770
:106AC000F1CF863009F44BC0873009F66A30C1F641
:106AD00080E0BECF882319F1813009F0B8CF633050
:106AE00079F688A1826188A381E0E0CFCE01825B44
:106AF0009F4F0E94A911CE018E599F4F0E94A9114C
:106B0000CE018C599F4F0E94A911D5CF633049F314
:106B1000643081F0113009F0B3CF80E099CF61305B
:106B200009F495CF623009F0ABCF88A1826088A3C9
:106B300081E0BCCF88A1886188A381E0B7CF6430B1
:106B400009F485CF653030F3653009F4ABCF66309A
:106B500009F096CF88A1816088A381E0A7CF673034
:106B600049F3683090F4663009F08ACF80E070CF46
:106B70006A3091F02FEF3FEF88A1886188A381E010
:106B80002115310509F492CF0AC0862F8950823031
:106B900008F076CF80E05CCF20E030E0EDCFC90197
:106BA000DF91CF911F910895CF93DF93EC0162E0C5
:106BB0000E9412358B89823031F08B89843069F4E0
:106BC00080E090E00CC040E050E060E070E0CE017A
:106BD0008C599F4F0E941112F0CF8FEF9FEFDF91E2
:106BE000CF910895CF93DF93EC018B89882339F0FF
:106BF000C05ADF4F88E497E2998388830FC061E031
:106C0000CE010E94123540E050E060E070E0CE011D
:106C10008E599F4F0E94111280E090E0DF91CF913A
:106C20000895CF93DF93EC01FB0180899189A289BC
:106C3000B3898C8B9D8BAE8BBF8BFA018081918148
:106C40009F8F8E8FFB0184859585A685B7858A8F5A
:106C50009B8FAC8FBD8FFA0184819581A681B7810E
:106C6000082E8B2FB02D092E9A2FA02D8CAF9DAF03
:106C7000AEAFBFAF8DA79EA7AFA7B8ABC05CDF4FCD
:106C80000196A11DB11D88839983AA83BB83C0543B
:106C9000D04086859785082E892F902D9EAB8DAB91
:106CA000FB01648575858685978540E050E00E94EC
:106CB000B72CFC01892BF1F00784F089E02D838942
:106CC00094898897FE01EE5AFF4F2081318121156A
:106CD000310561F4918380832081318189899A898A
:106CE0002817390738F43A8B298B04C08217930789
:106CF00098F7F0CFDF91CF9108950F931F93CF9323
:106D0000DF93EC01FC01E65AFF4F808191810196EF
:106D10009183808301970897B8F4E8ADF9AD0081BD
:106D200011814A8D5B8D6C8D7D8D9F0186E00E9467
:106D3000113F892B89F40E940D0FC25ADF4F7983CE
:106D4000688380E090E011C06CE477E2CE010E949D
:106D5000E4338FEF9FEF09C019AF08AF62E477E229
:106D6000CE010E94E4338FEF9FEFDF91CF911F910F
:106D70000F9108958F929F92AF92BF92CF92DF9220
:106D8000EF92FF920F931F93CF93DF936C01FB0160
:106D9000BA01E084F184028513850E2CE12E102DBA
:106DA0000F2CF02E002DEC0189A59AA5ABA5BCA552
:106DB0008E159F05A007B10730F488A1886188A3CC
:106DC00080E090E0E5C0E6012DA13EA14FA158A5CD
:106DD000E216F3060407150709F481C0E216F3066C
:106DE0000407150708F4A5C0E216F3060407150703
:106DF00009F48DC0E6011FAAEDA2FEA20FA318A7F9
:106E000086859785082E892F902DF60196AB85AB48
:106E1000CC5ADF4F88819981AA81BB810097A10557
:106E2000B10509F089C0188219821A821B82F60105
:106E3000C0ADD1AD2097C9F42EE530E0C20ED31E0F
:106E4000E60119821882E2EAFFEFCE0EDF1E3DC096
:106E500088819981F60191AF80AFCE010E944D25C6
:106E6000F601C0ADD1AD209739F3EB85FC852481C7
:106E7000358146815781022E252F502D032E342F28
:106E8000402D89899A89AA27BB27280F391F4A1FB5
:106E90005B1F8585992783709070892B21F02F5F68
:106EA0003F4F4F4F5F4FE216F3060407150780F67A
:106EB0000E940D0F2EE530E0C20ED31EE60179834D
:106EC0006883E2EAFFEFCE0EDF1E2AE530E0C20E55
:106ED000D31EE6011982188280E090E059C08480B8
:106EE0009580A680B780082C8B2CB02C092C9A2C6E
:106EF000A02C8DA59EA5AFA5B8A988159905AA05B2
:106F0000BB0568F188169906AA06BB06F9F0E601EA
:106F100088AD99AD892B69F0672B59F48585992740
:106F200083709070892B29F48FA98F5F8FAB83308A
:106F300038F580E090E02CC08E159F05A007B107C2
:106F400008F071CFC6010E944D3D6DCF89A99AA965
:106F5000ABA9BCA9E816F9060A071B07C0F286858B
:106F60009785082E892F902DE6019EAB8DAB8DA6BF
:106F70009EA6AFA6B8AAE9AAFAAA0BAB1CAB2ECF65
:106F80001FAAC6010E947D36892B99F28FEF9FEFD1
:106F9000DF91CF911F910F91FF90EF90DF90CF90F5
:106FA000BF90AF909F908F900895CF93DF93CDB710
:106FB000DEB72C970FB6F894DEBF0FBECDBF80E2D0
:106FC0000E94F60D3324339423E0231508F4FEC009
:106FD00048EC50E060E070E08BE793E00E94111213
:106FE000892B09F0F3C0E0917903F0917A03F887D7
:106FF000EF8310927A03109279031092D2021092CA
:10700000D102EF2B01F3EF81F885A385B485878149
:107010009085FC0124853585468557856D917C9149
:107020001197FD01828193810E942D265C01AF8121
:10703000B8854D905C901197892B09F4C2C0FD0171
:1070400085859685459708F45DC0C384D484B601D0
:107050006C5E7F4FD501AE5ABF4FFB014081442388
:10706000B1F09B012C193D09EF81F8858585968546
:107070002817390764F4413051F1423059F1FB01CE
:107080008181680F711DFB014081442351F7F60196
:107090001585F5018389853009F43FC0863008F0F5
:1070A00051C0823009F4D1C1833008F04DC188232A
:1070B00009F487C0813009F480C08F8198850E94CF
:1070C0004D2558864F82452809F09DCF7CCF6F5FB4
:1070D0007F4FC3CFFB0182819927382F22278381DD
:1070E0009927282B392B022E232F302D8D919C91FF
:1070F00011972817390718F411963C932E936C5F5B
:107100007F4FABCFEF81F885C384D484F60115851A
:10711000F5018389853009F0C1CF812F992782FD40
:10712000A8C181FD4EC084FFC8CFEF81F885418999
:107130005289B601C5010E94BA368F8198850E9496
:107140004D25BFCF883009F459C1893008F0B9C046
:10715000863009F4BFC1873009F0AFCF812F99275E
:1071600082FD91C181FD2DC084FFA7CFEF81F885FD
:1071700041895289B601C5010E94BA36F50121A59F
:1071800032A543A554A585A196A1A7A1B0A528170E
:1071900039074A075B0709F090CF2CE530E0A20ED3
:1071A000B31ED5011D921C92E4EAFFEFAE0EBF1E86
:1071B0006AE0C5010E94123580CF1671123009F4C1
:1071C00028C28F8198850E9487317BCFE090BC02D6
:1071D000F090BD02E114F10409F571C0F70180AD32
:1071E00091AD892B41F08701025A1F4FD8018D9133
:1071F0009C91892B89F5F70183898A30E9F083898D
:107200008930D1F0F7018389833009F43FC0D70179
:10721000ED90FC90E114F10409F451C0F70180A154
:1072200084FFDCCF886080A340E050E060E070E045
:10723000C7010E942232D2CFF701E45AFF4F80816A
:1072400091810196918380830197099700F3C7018B
:107250000E94702B3324B7CE0E940D0FF8012081BD
:107260003181621B730B28E530E0E20EF31ED7017B
:107270002D913C91E8EAFFEFEE0EFF1E261737072F
:1072800008F0B9CFC7010E947D36B5CFD701A45A07
:10729000BF4F8D919C911197019611969C938E935F
:1072A00001978D9708F4B3CF81E0838B1D921C92D8
:1072B000D701ED90FC90E114F10409F0AFCF332435
:1072C00082CE893009F0F9CE012F112702FDDBC0F3
:1072D00001FD77CF04FFF1CEEF81F8854189528916
:1072E000B601C5010E94BA36EF81F885818992897D
:1072F000892B09F492C2BF01C5010E94A834C501BF
:10730000825B9F4F0E94B41100FFDBCEF501E05C71
:10731000FF4F80819181A281B3810196A11DB11D92
:1073200080839183A283B3832CE530E0A20EB31E49
:10733000D5011D921C92E4EAFFEFAE0EBF1E6AE07B
:10734000C5010E941235BDCE833009F417C18430C7
:1073500009F0B3CEF50105A8F6A9E02DFA83E9837B
:10736000F50125A136A147A150A52B833C834D8370
:107370005E83812E992482FC3CC281FEA4C1F60169
:1073800084819581A681B781082E8B2FB02D092E7F
:107390009A2FA02DF50124AD35AD46AD57AD82171E
:1073A0009307A407B50709F433C28F8198850E941B
:1073B0008731F50183898430E1F489819A819C01C8
:1073C0004427552785A996A9AA27BB272817390737
:1073D0004A075B0770F085A196A1A7A1B0A52B81F4
:1073E0003C814D815E81281739074A075B0708F009
:1073F00068CEC501CA960E94A91163CE812F992734
:1074000082FD41C081FDDDCE84FF57CEEF81F8853E
:1074100041895289B601C5010E94BA368F8198858B
:107420000E944D25F50121A532A543A554A585A1AE
:1074300096A1A7A1B0A5281739074A075B0709F04D
:1074400040CEC5010E94702B3CCE812E992490E144
:10745000692E712C6820792084FCB9C082FE1BC083
:10746000672809F42ACE6DE477E2C5010E94E4336F
:1074700024CE8F8198850E944D2566E477E2C50170
:107480000E94E4331ECE8F8198850E944D25C50150
:107490000E94702B16CE81FE10CEEF81F885678199
:1074A0007085A601C5010E941136672809F4ABC199
:1074B000EF81F88541895289B601C5010E94BA362B
:1074C00064E0C5010E941235C5018C599F4F0E948E
:1074D000B411F3CD012F112702FDD5CF01FD71CEDF
:1074E00004FFEBCDEF81F88541895289B601C501D2
:1074F0000E94BA36F50121A532A543A554A585A160
:1075000096A1A7A1B0A5281739074A075B0709F478
:107510004DC2EF81F88581899289892B09F482C156
:10752000BF01C5010E94A834C501825B9F4F0E9424
:10753000B41100FFC6CDF501E05CFF4F8081918161
:10754000A281B3810196A11DB11D80839183A28385
:10755000B3832CE530E0A20EB31ED5011D921C9220
:10756000E4EAFFEFAE0EBF1EF5018389893009F40E
:10757000E6CE67E0C5010E941235A3CD812E992485
:1075800082FE58C022E630E0A20EB31ED5018D91D6
:107590009C91EEE9FFEFAE0EBF1E892B09F447C1A7
:1075A00061E0C5010E9412358F8198850E944D25AA
:1075B0002EE530E0A20EB31ED5011D921C92E2EA28
:1075C000FFEFAE0EBF1EC5010E9431277ACDF60136
:1075D0006085718582859385062E692F902D072EF3
:1075E000782F802DF501E1A4F2A403A514A521A113
:1075F00032A143A154A12F5F3F4F4F4F5F4F0E94D5
:10760000203D892B09F02ACF8F8198850E948731F0
:1076100058CDEF81F88567817085A601C5010E946C
:10762000113663E0C5010E9412358F8198850E9452
:107630004D2547CD81FCC5CD84FE3FCDF60160854B
:10764000718582859385062E692F902D072E782FC0
:10765000802DF501E1A4F2A403A514A525A136A16E
:1076600047A150A52F5F3F4F4F4F5F4F0E94203DD6
:10767000892B09F4A6CDEF81F88541895289B6019D
:10768000C5010E94BA36EF81F88581899289892BDC
:1076900009F487C1BF01C5010E94A83480FE72C1F0
:1076A000F501E05CFF4F80819181A281B381019659
:1076B000A11DB11D80839183A283B38365E0C501C1
:1076C0000E941235FECC84FEA3C0EF81F88541896B
:1076D0005289B601C5010E94BA36F601448155812E
:1076E00066817781DB01CA01082E8B2FB02D092E10
:1076F0009A2FA02D30E4632E712C6A0C7B1CF301B1
:10770000C080D180E280F380C816D906EA06FB0665
:1077100008F093C0EF81F88581899289892B09F45B
:107720002CC1F501E05BFF4FE080F1806F01E114B7
:10773000F10409F44BC08A019B01002E032F302D68
:10774000012E122F202DF701A385B485FD01848120
:107750009581A681B781082E8B2FB02D092E9A2FE7
:10776000A02D081719072A073B0708F429C180171D
:107770009107A207B30719F500C18A019B01002EEA
:10778000032F302D012E122F202DF701A385B48554
:10779000FD0184819581A681B781082E8B2FB02DA4
:1077A000092E9A2FA02D081719072A073B0708F45E
:1077B00007C1081719072A073B0709F4DEC067014C
:1077C000D701ED90FC90E114F104B9F6EF81F88552
:1077D000D601ED93FC9311821082F50180A188619E
:1077E00080A340E050E060E070E0C5010E942232DA
:1077F000E0CD8F8198850E944D2566E477E2C50132
:107800000E94E433D6CD63E0C5010E94123555CC09
:107810008F8198850E944D25CCCD8F8198850E94BF
:107820004D2572CD8F8198850E944D2582CE6DE4C5
:1078300077E2C5010E94E433B7CE042E472F702DA6
:10784000052E562F602DC416D506E606F70679F1EB
:10785000F50180A1886180A3E259FF4F8081918169
:10786000A281B3810196A11DB11D80839183A28362
:10787000B3838F8198850E944D2540E050E060E001
:1078800070E0C5010E94223280FE93CDF301808119
:107890009181A281B3810196A11DB11D8083918345
:1078A000A283B38365E0C5010E94123582CDEF81CA
:1078B000F88581899289892B09F47DC0BF01C501B2
:1078C0000E94A83420E5822E912C8A0C9B1CD401A6
:1078D0006D917C916115710509F43FC0FB01038432
:1078E000F485E02DF887EF83248135814681578127
:1078F000DA01C901082E8B2FB02D092E9A2FA02D49
:1079000089879A87AB87BC87D301CD90DD90ED90B6
:10791000FC9089859A85AB85BC85C816D906EA0690
:10792000FB06D8F0DB018D919C91F401918380835B
:10793000022E252F502D032E342F402D2C153D05C2
:107940004E055F0591F0CB010E944D25D4016D914C
:107950007C916115710509F0C1CFC501825B9F4F14
:107960000E94B411812E99248FCFC5010E94A834A2
:10797000EF81F8858585182BAACF8F8198850E9485
:107980004D252BCF64E0C5010E941235C5018E59EB
:107990009F4F0E94B411C5018C599F4F0E94B41192
:1079A00090CB8F8198850E944D2578CE69E0C501E6
:1079B0000E941235AECD8F8198850E944D2564CFEF
:1079C000EF81F885D601ED93FC93F182E08205CF3B
:1079D000CF93DF93EC01892B79F00E947E0E8B8987
:1079E000853068F0853019F18B30C0F0C05ADF4F18
:1079F00089E497E2998388838FEF9FEF1EC08330DD
:107A000038F066E0CE010E94123580E090E015C0AB
:107A1000CE010E94702B80E090E00FC0C05ADF4F73
:107A200085E397E2998388838FEF9FEF06C068E034
:107A3000CE010E94123580E090E0DF91CF91089551
:107A4000EF92FF920F931F93E216F30604071507B8
:107A500070F06217730784079507C0F020E030E0EC
:107A6000E616F7060807190770F4C90111C02617B2
:107A700037074807590750F020E030E06E157F05C2
:107A80008007910790F321E030E0EFCF80E090E0B5
:107A90001F910F91FF90EF9008950F931F93CF9335
:107AA000DF938C01EC01C25ADF4F88819981892BC9
:107AB00019F10E940D0F28813981621B730B9B0104
:107AC000F801E85AFF4F80819181880F991F280F94
:107AD000391F220F331F220F331F87E0203D380745
:107AE00028F468EC70E07183608306C0C9016AE025
:107AF00070E00E945B4AF7CFDF91CF911F910F9109
:107B00000895EF92FF920F931F937C010027112796
:107B1000FB0142305105A0F081819927982F8827D9
:107B200020813327822B932BAA27BB27E80EF91E2F
:107B30000A1F1B1F3296425050404230510560F7D9
:107B4000452B61F08081E80EF11C011D111D06C05E
:107B500000271127E80EF91E0A1F1B1FC801AA27BC
:107B6000BB270097A105B10599F7C7011F910F9198
:107B7000FF90EF9008950E94813D80959095089523
:107B8000EF92FF920F93CF93DF93CDB7DEB72C9791
:107B90000FB6F894DEBF0FBECDBF69837A838B83A7
:107BA0009C832D833E834F83588719860A87FC86E2
:107BB000EB864CE050E0BE016F5F7F4F80E090E0CD
:107BC0000E94813DAA27BB27BC01CD012C960FB690
:107BD000F894DEBF0FBECDBFDF91CF910F91FF9024
:107BE000EF9008959093D4028093D30208952F923A
:107BF0003F924F925F926F927F928F929F92AF923D
:107C0000BF92CF92DF92EF92FF920F931F93CF9389
:107C1000DF93CDB7DEB723970FB6F894DEBF0FBE64
:107C2000CDBF1C015B01FB010780F085E02DFB83CC
:107C3000EA832081822F807F803421F0C5010E9459
:107C40004D25D6C086819781082E892F902D9F7350
:107C5000892BA1F74091D3025091D40241155105CF
:107C600059F06485758586859785FA010995892B74
:107C700029F7EA81FB8120812F702983EA81FB812A
:107C80006088718882889388F10147845088FFEF6B
:107C90006F16FFEF7F06FFEF8F06FFEF9F0671F174
:107CA000F201278130854185528521153105410535
:107CB000510509F45CC087859089A189B2898F3FFD
:107CC000FFEF9F07FFEFAF07FFEFBF0749F08629E0
:107CD0009729A829B9298F5F9F4FAF4FBF4F71F0E8
:107CE000611471048104910409F4A8CF621673062B
:107CF0008406950609F0A2CF60E001C061E0F98139
:107D00002F2F3327220F331F220F331FF501328706
:107D100021878A819B81820F931F94878387EA81C1
:107D2000FB8182819381082E892F902D821B930BDA
:107D3000F50196878587EA81FB818185863009F484
:107D40004DC0813109F451C0813009F442C066232D
:107D500009F074CF850120E030E040E050E062E0BF
:107D600083E00E944741892B09F468CF41C0EA8132
:107D7000FB818185813009F0BFCFD401C3018070C0
:107D80009070A0708030F0E09F07F0E0AF07FFEF49
:107D9000BF0709F4B1CF0097A105B10509F4ACCF35
:107DA000CC24DD24760100E010E020E030E0B401D6
:107DB000A301C1010E94802FF201278130854185F6
:107DC0005285211531054105510509F089CF60E043
:107DD00096CFB501C1010E946C400AC0662309F02C
:107DE0002DCFC5010E94804403C0C5010E94B34449
:107DF00023960FB6F894DEBF0FBECDBFDF91CF91B3
:107E00001F910F91FF90EF90DF90CF90BF90AF90B8
:107E10009F908F907F906F905F904F903F902F90AA
:107E200008954F925F926F927F928F929F92AF923E
:107E3000BF92CF92DF92EF92FF920F931F93CF9357
:107E4000DF93CDB7DEB72A970FB6F894DEBF0FBE2B
:107E5000CDBF182F4A015B01C90144E150E060E247
:107E60000E945B246C01009709F4FFC0FC01E780CD
:107E7000F08485E4F70180831182F6018185928583
:107E800025853685820F931F21893289820F931FA2
:107E9000082E892F902DF7019383828317821682F3
:107EA00080E480871187808A918AA28AB38AFFEF53
:107EB0008F16FFEF9F06FFEFAF06FFEFBF0609F437
:107EC00047C0AE014F5F5F4FC501B4010E94B72CA0
:107ED0003C01009709F4C6C0FC0107851089F80130
:107EE000858996890196968B858B0197082E892F17
:107EF000902DF70195838483F80187819085A18572
:107F0000B285F70184879587A687B787138612867F
:107F1000F601418552856781708580E090E00E947E
:107F2000BB3DF70193878287F8018081863009F491
:107F30006CC0873109F096C0F801A58DB68D960109
:107F400040E050E061E270E0C301FD010995ADC081
:107F500025E0422E512C4C0E5D1E46E050E06FEFA6
:107F600070E0C2010E941F4A00918D0210918E02A2
:107F70000115110569F486C080E090E0F8010081E8
:107F800011810115110509F490C0009709F08DC009
:107F9000F8018385833081F7F801A784B088F50163
:107FA000858996890196968B858B0197082E892F56
:107FB000902DF70195838483F50187819085A185B4
:107FC000B285F70184879587A687B78713861286BF
:107FD000F601418552856781708580E090E00E94BE
:107FE000BB3DF70193878287F5018081863009F4D4
:107FF0003FC0F501A58DB68D960140E050E061E2ED
:1080000070E0C801FD010995B9CF89819A81AB81E2
:10801000BC810097A105B105C1F587859089A1892B
:10802000B28988299929AA29BB298F5F9F4FAF4F11
:10803000BF4F71F185E0482E512C4C0E5D1E920110
:10804000B501A401C3010E947E42892BD9F4F80135
:10805000A58DB68D9601A20160E078E0C301FD0117
:10806000099523C0C6010E944D258FEF9FEF1DC0CB
:10807000A58DB68D9601A20160E078E0C801FD01F2
:1080800009957CCF80E090E010C04C015D01D2CF1B
:1080900095E0492E512C4C0E5D1E46E050E06FEFEE
:1080A00070E0C2010E941F4AD2CF2A960FB6F89400
:1080B000DEBF0FBECDBFDF91CF911F910F91FF901B
:1080C000EF90DF90CF90BF90AF909F908F907F9078
:1080D0006F905F904F9008950F931F93CF93DF930E
:1080E0008C01EB018D859E8589309105A8F04B852B
:1080F0005C859C01285030403A8B298BDA01189618
:10810000B88BAF8788E090E09E878D87FA018081E9
:10811000833031F0883059F1CE010E944D2544C0A2
:108120002D313105C8F3FD0181858630A9F7CA01DB
:1081300088569E4F2485358546855785FC0160818C
:108140007181828193810E942D26FC01892B21F36C
:108150008389823019F083898430F1F661E577E212
:10816000CF010E94E433CE010E944D251DC02F8116
:108170003885F9014485558566857785F801A78599
:10818000B089FD0187819085A185B285F901848739
:108190009587A687B7878FEF80879E0180E00E9432
:1081A000D940892B09F4B8CFDF91CF911F910F915E
:1081B0000895AF92BF92CF92DF92EF92FF920F930A
:1081C0001F935A016B018901F901E384F484F701DB
:1081D000808313821282F9014585568563857485F3
:1081E00080E090E00E94813DF801418952896785D5
:1081F00070890E94BB3DF701938382839801B60189
:10820000A50181E00E94113F1F910F91FF90EF9017
:10821000DF90CF90BF90AF9008956F927F928F9232
:108220009F92AF92BF92CF92DF92EF92FF920F9305
:108230001F93CF93DF93682E762E49015A01C60112
:1082400048E050E060E40E945B24009779F0EC0184
:10825000EB85FC85718284829582A682B7829C011F
:10826000B801A701862D0E94D94002C08FEF9FEF71
:10827000DF91CF911F910F91FF90EF90DF90CF9002
:10828000BF90AF909F908F907F906F9008956F9266
:108290007F928F929F92AF92BF92CF92DF92EF9296
:1082A000FF920F931F93CF93DF93682E762E490191
:1082B0005A01D801E801EF81F885E484F584068548
:1082C00017854CE150E060E8CD010E945B24EC0191
:1082D000892BD9F0AF85B889EF81F88584E10190C9
:1082E0000D928150E1F7EF85F8897496AB85BC85D6
:1082F00088E00D9001928150E1F76E01A501940193
:10830000672D862D0E940D4102C08FEF9FEFDF91F8
:10831000CF911F910F91FF90EF90DF90CF90BF9082
:10832000AF909F908F907F906F900895CF93DF9341
:10833000EC01EF89F88D3097C1F082819381A4819F
:10834000B581481759076A077B0751F40EC082812F
:108350009381A481B58184179507A607B70729F0F3
:108360000190F081E02D309791F7CF01DF91CF910F
:1083700008950F931F93CF93DF93FC01C789D08D8E
:108380002097F1F08C01095E1F4F06C08E01099005
:10839000D881C02D2097A1F08C8580FFF7CFCE012A
:1083A0000E960E94721188819981F80191838083D1
:1083B000CE010E945A49F801C081D181209761F70E
:1083C000DF91CF911F910F910895CF93DF930E947A
:1083D000800F2091D5023091D6024091D702509162
:1083E000D802621B730B840B950B6C3371058105EE
:1083F000910508F440C00E94800F6093D5027093ED
:10840000D6028093D7029093D802C0918D02D0916A
:108410008E02209731F42FC00990D881C02D20976B
:1084200051F18B858330C1F7AF85B8891097A1F3DF
:108430008C91863089F7FD014789508D4115510592
:1084400059F320E0FA01948592FD08C085858F5F7D
:1084500085878150893010F091609487292BFA012B
:10846000408151814115510569F720FFD5CFCD01DC
:108470000E94B941D1CFDF91CF910895AF92BF92C1
:10848000CF92DF92EF92FF920F931F93CF93DF93E0
:108490005C017A018B0169010E94E54180E190E075
:1084A0000E945D49FC01892BE9F080E1DF011D920A
:1084B0008A95E9F7E282F38204831583C114D1041B
:1084C00051F0EF012696D60186E00D900992815079
:1084D000E1F782E08487E5018F89988D918380831D
:1084E000F88FEF8BCF01DF91CF911F910F91FF900C
:1084F000EF90DF90CF90BF90AF9008952F923F9272
:108500004F925F927F928F929F92AF92BF92CF9243
:10851000DF92EF92FF920F931F93CF93DF93CDB72C
:10852000DEB724970FB6F894DEBF0FBECDBF1C0197
:108530005A016B013A832983FC01478450880E94C9
:10854000E541B601A501C2010E9496419C838B833F
:10855000892B09F46EC08824992421E0722E94EFAF
:10856000E92E91E0F92E012D112DEB81FC818485FE
:1085700081FD27C07A949FEF7916B1F1811491049F
:1085800039F0B401C1010E94F743892B09F043C0BF
:10859000B801A7018B819C810E960E941112B60131
:1085A000A501C2010E9496419C838B83892BE1F037
:1085B000EE0CFF1C001F111FEB81FC81848581FFE5
:1085C000D9CFDF0129813A812A5F3F4FFD018385A1
:1085D000F90182939F01119789819A81E817F90720
:1085E000A9F700E010E002C00FEF1FEF8114910423
:1085F00009F440C0C4010E944D2501151105D1F1B7
:10860000EB81FC813097B1F1848581608487C20160
:108610000E94B9412FC0B601A501C2010E94964136
:10862000FC01892B19F0848581FF1DC00FEF1FEF1E
:1086300021C020E030E0B601A501C2010E943E4207
:108640009C838B83892B91F320E030E0B601A50158
:1086500081E090E00E9424444C01892B09F07DCFF9
:10866000EB81FC81848581608487C2010E94B941CD
:108670000FEF1FEFC80124960FB6F894DEBF0FBEB0
:10868000CDBFDF91CF911F910F91FF90EF90DF90C1
:10869000CF90BF90AF909F908F907F905F904F90C2
:1086A0003F902F900895CF92DF92EF92FF920F9319
:1086B0001F93CF93DF93EC017A018B0169018F85C2
:1086C00098890E949641FC01892BA9F0848582FF3C
:1086D00005C0CF010E960E94A91114C01586EF01A6
:1086E0002696D60186E00D9009928150E1F78485A7
:1086F00082608487EECF9601B801A7018F859889A3
:108700000E943E42DF91CF911F910F91FF90EF9019
:10871000DF90CF900895CF92DF92EF92FF920F9368
:108720001F93CF93DF937C018B01FB01C781D08521
:1087300088819981082E892F902D019709F04BC0CF
:108740008A819B81082E892F902D8050984009F0B6
:1087500042C08C81863009F03EC08D81843009F0A2
:108760003AC0F701A785B089288D398D4A8D5B8D78
:10877000FD0187819085A185B285281739074A07B1
:108780005B0749F588E0C82ED12CCC0EDD1E4E8546
:108790005F85688979899601C7010E9453438E815C
:1087A0009F81082E892F902D0197A9F44E855F8512
:1087B00068897989960182E090E00E942444EC0166
:1087C000009749F0BC01C7010E94F743892B19F4B7
:1087D000CE010E944D25C8010E944D25DF91CF9109
:1087E0001F910F91FF90EF90DF90CF9008950F931E
:1087F0001F93CF93DF938C01AB01FB01C781D08521
:10880000FC0127853089DE011896F901319686E052
:1088100001900D928150E1F7F90187819085A18542
:10882000B2858E879F87A88BB98B6296A58DB68DF2
:108830009A01AE0166E078E0C801FD010995DF917B
:10884000CF911F910F9108958F929F92AF92BF92F7
:10885000CF92DF92EF92FF920F931F93CF93DF930C
:108860008C014A015B0169014CE150E060E280E06B
:1088700090E00E945B247C01009709F433C0FC0166
:10888000C781D08581E090E0082E892F902D9983B3
:10889000888380E098E0082E892F902D9B838A831F
:1088A00086E08C8384E08D83002E012F102D1F83A2
:1088B0000E83C114D10469F0DE015296F60186E000
:1088C00001900D928150E1F7888E998EAA8EBB8E11
:1088D00009C046E050E06FEF70E0CE0142960E9482
:1088E0001F4AF2CFC701DF91CF911F910F91FF90E7
:1088F000EF90DF90CF90BF90AF909F908F900895B2
:10890000CF93DF93FC01A385B485ED018C8582951F
:108910008F709927880F991F880F991F2585368595
:10892000281B390B328B218B232B61F08C85829590
:108930008F709927880F991F880F991F8A0F9B1F87
:10894000908B8787ED018C8582958F709927880F92
:10895000991F880F991F96878587CF010E942F3412
:10896000DF91CF910895EF92FF920F931F93CF93D2
:10897000DF937C01162FEC01EB85FC853896F88B94
:10898000EF8738978D859E8508979A8B898B88E02D
:1089900090E09E878D87828193810E942445EC011F
:1089A000892BB9F12A853B8521153105B1F48C81DC
:1089B0009D81009711F00E944D25FD82EC82F70108
:1089C00081899289998788878E819F81892BA9F1D6
:1089D000CE0106960E94B41130C048855985F70132
:1089E00061897289CA01860F971F28173907F0F02D
:1089F000EC81FD81309711F41DC0FC0180819181D3
:108A00000097D9F7F182E082460F571F59874887B0
:108A1000DBCF112359F4870120E030E040E050E043
:108A200063E083E00E944741892B39F4C7010E942B
:108A30004D2503C0FD82EC82E7CFDF91CF911F91DE
:108A40000F91FF90EF9008959C01E0917D03F091CC
:108A50007E03309781F0828193812817390731F4A2
:108A60000DC0828193818217930741F00190F081BC
:108A7000E02D3097B1F780E090E00895CF010895A0
:108A8000FC01DA01892B19F48FEF9FEF08956250F2
:108A90007041D1F7452BC1F322303105A9F78D91F3
:108AA0009C919387828780E090E00895FC01DA0131
:108AB000892B19F48FEF9FEF089562507041D1F721
:108AC000452BC1F322303105A9F7828593858D931B
:108AD0009C9380E090E00895CF93DF93EC01E091C8
:108AE0007D03F0917E03309769F0E817F90721F4D0
:108AF0000CC0CE17DF0759F0DF010190F081E02DA7
:108B00003097B9F78FEF9FEF1AC0ADE7B3E08881D8
:108B100099818D939C93EC81FD81309759F08081F0
:108B200091819D838C83CF010E944D25EC81FD8135
:108B30003097A9F7CE010E94610C80E090E0DF91B0
:108B4000CF9108956F927F928F929F92AF92BF9232
:108B5000CF92DF92EF92FF920F931F93CF93DF9309
:108B60003C015A016B014901A70160E880E090E0F7
:108B70000E945B24EC01892BA1F0A701B8018F852D
:108B800098890E94164A8E019401B601A501C3017D
:108B90000E9498468C01892B31F4CE010E944D250C
:108BA00002C00FEF1FEFC801DF91CF911F910F910E
:108BB000FF90EF90DF90CF90BF90AF909F908F90FD
:108BC0007F906F900895CF93DF93EC01892B51F53F
:108BD00040917D0350917E03C0916802D09169025B
:108BE000219611F4C0E0D0E19E01022E232F302DFA
:108BF0004115510599F0FA018281938182179307FB
:108C000079F3DA010D90BC91A02D109739F0FD0198
:108C1000828193812817390719F3F4CFD093690221
:108C2000C09368028CE090E00E94E30CFC01892B69
:108C300079F00C2ECD2FD02DD383C28380917D036C
:108C400090917E0391838083F0937E03E0937D0374
:108C5000CF01DF91CF9108954F925F926F927F92F3
:108C60008F929F92AF92BF92CF92DF92EF92FF923C
:108C70000F931F93CF93DF935C014B013A012901BE
:108C8000FC01C481D5812097A1F188819981F501EA
:108C900095838483EF81F88584859585A685B7853E
:108CA000F40180839183A283B383EB85FC8580816B
:108CB0009181082E892F902DF30191838083E9887B
:108CC000FA8897010E151F0590F0F50180859185B2
:108CD000821B930B918780876F857889A701C201DA
:108CE0000E94164ACE010E944D25A7010FC07801AF
:108CF000ECCFB701A60106960E941112F501C481BE
:108D0000D581209709F0C1CF40E050E0CA01DF9142
:108D1000CF911F910F91FF90EF90DF90CF90BF9078
:108D2000AF909F908F907F906F905F904F9008953D
:108D30004F925F926F927F928F929F92AF92BF926B
:108D4000CF92DF92EF92FF920F931F93CF93DF9317
:108D5000CDB7DEB724970FB6F894DEBF0FBECDBFF8
:108D60002C013A014B017901C80148E050E060E470
:108D70000E945B245C01009709F456C0FC01C38487
:108D8000D484F20182819381F601918380830E2C39
:108D9000EF2CF02CF382E282F501858596852189FE
:108DA0003289820F931F082E892F902DF60195830B
:108DB0008483AE014F5F5F4FC401B3010E94B72CA3
:108DC000FC01892BA1F10784F089E02D8781908532
:108DD000A185B28589839A83AB83BC83F601178210
:108DE0001682E480F58069817A818B819C8101E122
:108DF000A40193010E94C03DDC01CB0148E050E09A
:108E0000B6010E94813DF5014189528967857089CB
:108E10000E94BB3DF601978386839501B401A301AF
:108E200081E10E94113F08C08FEF9FEF05C01982BA
:108E30001A821B821C82D2CF24960FB6F894DEBF12
:108E40000FBECDBFDF91CF911F910F91FF90EF909B
:108E5000DF90CF90BF90AF909F908F907F906F905A
:108E60005F904F900895CF93DF93EC01AA81BB816F
:108E7000109731F0ED01ED89FE89CD01099503C010
:108E8000EB85FC850995DF91CF910895EF92FF92D4
:108E90000F931F93CF93DF938C01892B71F0C0E068
:108EA000D0E0EAE6F2E0808191810817190779F0B5
:108EB00021963296C830D105B1F789E090E09093C1
:108EC000800380937F032FEFE22EF22E17C0F8016C
:108ED000808191810E946A49892B61F4EE24FF24EC
:108EE000C8010E945A49CC0FDD1FC659DD4F1982B7
:108EF000188204C09FEFE92EF92EF2CFC701DF914F
:108F0000CF911F910F91FF90EF900895EF92FF92F4
:108F10000F931F93CF93DF937C01CB010E94F44703
:108F20008C018FEF0F3F1807D9F08091700290915C
:108F30007102892BC1F084E090E0E2E7F2E0EC01FD
:108F400080819181892B89F0CE01019632968830FB
:108F50009105A9F787E190E09093800380937F03C8
:108F600080E090E025C0C3E0D0E087E090E00E9480
:108F70005D49DC01CC0FDD1FFE01E659FD4FB183D9
:108F8000A083109771F01196FC92EE92FD0113836D
:108F90000283148216821582C659DD4F8881998119
:108FA00007C08CE090E09093800380937F03F4CF20
:108FB000DF91CF911F910F91FF90EF900895FC01E9
:108FC00040E050E060E070E0808191810E94FB49C8
:108FD000892B19F480E090E008958FEF9FEF0895BA
:108FE000FC01808191810895FC018081823769F0C4
:108FF000873701F1813609F186E190E09093800393
:1090000080937F038FEF9FEF089580E090E4319687
:109010002081222351F02B3249F0223669F79F7BC1
:109020009068319620812223B1F708958E7F826067
:109030009360EDCF81E093E4EACF88E091E4E7CF5D
:10904000CF92DF92EF92FF920F931F93CF93DF9314
:109050006C01CB010E94F4477C018F5F9F4F71F13F
:109060008091700290917102892BC1F084E090E0B0
:10907000E2E7F2E0EC0180819181892B89F0CE0159
:109080000196329688309105A9F787E190E0909398
:10909000800380937F0380E090E030C0C3E0D0E0A5
:1090A00087E090E00E945D498C01CC0FDD1FC6591E
:1090B000DD4F198308830115110519F480E090E054
:1090C0001DC0B701C6010E948049F80191838083C9
:1090D0008F5F9F4F59F0E881F981F382E282148219
:1090E000E881F98116821582CF0108C088819981B3
:1090F0000E945A491982188280E090E0DF91CF9156
:109100001F910F91FF90EF90DF90CF900895CF9334
:10911000DF93CDB7DEB721970FB6F894DEBF0FBE51
:10912000CDBFFC01848183FF05C0877F8483858157
:10913000968110C041E050E0BE016F5F7F4F80819B
:1091400091810E94E949019719F08FEF9FEF02C0CA
:109150008981992721960FB6F894DEBF0FBECDBF47
:10916000DF91CF910895EF92FF920F931F93CF93CA
:10917000DF93FC018B01E9016230710540F0CA0107
:10918000869FA001879F500D969F500D11248C81C2
:1091900083FD21C0EE24FF24BF01888199810E94B4
:1091A000E949BC01892B69F48C8180628C836E0D46
:1091B0007F1D02301105C8F0CB01B8010E945B4A47
:1091C00014C09FEF6F3F790791F78C8180618C838A
:1091D00060E070E0ECCF877F8C838D81819341507C
:1091E000504081E0E82EF12CD7CFCB01DF91CF9119
:1091F0001F910F91FF90EF900895FB01248123FFB1
:1092000003C08FEF9FEF08953FEF8F3F930721F04B
:10921000968385832860248308950F931F93CF93AB
:10922000DF93CDB7DEB721970FB6F894DEBF0FBE40
:10923000CDBF8C01FB01898341E050E0BE016F5F2F
:109240007F4F808191810E94FB49019711F00FEFC0
:109250001FEFC80121960FB6F894DEBF0FBECDBF39
:10926000DF91CF911F910F910895CF93DF93EB0181
:10927000F9016230710540F09A01269FA001279FF5
:10928000500D369F500D1124BC01808191810E94A8
:10929000FB49BC01181619063CF4C230D10530F068
:1092A000BE010E945B4A02C060E070E0CB01DF912A
:1092B000CF9108950E94610C08950E94E30B9C01D8
:1092C000892B31F48CE090E09093800380937F03AE
:1092D000C9010895CF93DF93EC01EA81FB813097B8
:1092E00029F0078CF0A1E02D099507C0EF81F885E2
:1092F00040E050E060E070E00995DF91CF91089583
:10930000CF92DF92EF92FF920F931F93CF93DF9351
:10931000CDB7DEB729970FB6F894DEBF0FBECDBF2D
:109320006C017B01DC012C912223B1F12A33A1F1E4
:109330008C01CE010196FC01AE01475F5F4F208397
:109340000F5F1F4F302F3C19D8012C91222331F091
:109350002A3321F03196E417F50789F7E32FFF2729
:10936000E80FF91F10820E949112DC01892BD1F0C5
:10937000F80180818A3361F060E070E0FD01058DC5
:10938000168D20E030E0A701CD01F801099512C04B
:10939000B8016F5F7F4FF2CF8601E0E0F0E0CE01D1
:1093A0000196DECF82E090E09093800380937F036C
:1093B0008FEF9FEF29960FB6F894DEBF0FBECDBF9B
:1093C000DF91CF911F910F91FF90EF90DF90CF90A1
:1093D0000895CF93DF93EC01EA81FB81309729F068
:1093E0000788F08DE02D099503C0ED81FE81099578
:1093F000DF91CF910895CF93DF93EC01EA81FB8158
:10940000309729F0018CF28DE02D099503C0EF8192
:10941000F8850995DF91CF910895FB01DC0102C029
:1094200005900D9241505040D8F70895FB01DC01A2
:1094300002C001900D9241505040D8F70895DC01D0
:1094400001C06D9341505040E0F70895FB01DC01ED
:109450008D910190801911F40020D1F7990B089596
:10946000629FD001739FF001829FE00DF11D649F08
:10947000E00DF11D929FF00D839FF00D749FF00D94
:10948000659FF00D9927729FB00DE11DF91F639F35
:10949000B00DE11DF91FBD01CF0111240895991BE5
:1094A00079E004C0991F961708F0961B881F7A95DB
:1094B000C9F780950895AA1BBB1B51E107C0AA1FDD
:1094C000BB1FA617B70710F0A61BB70B881F991F65
:1094D0005A95A9F780959095BC01CD010895A1E218
:1094E0001A2EAA1BBB1BFD010DC0AA1FBB1FEE1F1E
:1094F000FF1FA217B307E407F50720F0A21BB30B69
:10950000E40BF50B661F771F881F991F1A9469F7E4
:1095100060957095809590959B01AC01BD01CF0140
:109520000895E199FECFBFBBAEBBE09A11960DB294
:109530000895E199FECFBFBBAEBB0DBA11960FB631
:0A954000F894E29AE19A0FBE089534
:10954A004E75744F532D4254001A0C0103240C0318
:10955A00140180030C00130CF80A0407090407011C
:10956A000C04060D041730303030051000722B62DF
:10957A00007561727430003139322E3136382E312D
:10958A002E313030003235352E3235352E323535E2
:10959A002E300065746830007263760000069830D9
:1095AA0000350065746865726E75740069646C656F
:1095BA00006D61696E00FF00000000A414000075D0
:1095CA006172743000000000050000000000A00174
:1095DA00C81E4B1F5C2354234C236321E221E41E43
:1095EA000000000000000000000000000000000071
:1095FA000000000000000000000000000000000061
:10960A000000000000000000000000000000000050
:10961A000000000000C918B618311733170317F5F0
:10962A001628186918F0170E16B8172B1697173C34
:10963A00167F1646165D17DD160000657468300041
:10964A0000000000030000001C0296021F1B00001D
:10965A0000000000000000000000000006000000FA
:10966A00000000000000000000000000000000DC14
:10967A000500000000F72E7B1B242F00000000EEDF
:10968A0018000000005C19727869350000000000BB
:10969A00451D00103235352E3235352E3235352EF0
:1096AA003000746370736D00001001000200030043
:0A96BA0000000000000000000000A6
:00000001FF
